:100000000C94C3050C94EB050C94EB050C94EB05D8
:100010000C94EB050C94EB050C94EB050C94EB05A0
:100020000C94EB050C94EB050C94E2180C944B1912
:100030000C94EB050C94EB050C94EB050C94EB0580
:100040000C94EB050C94EB050C94EB050C94EB0570
:100050000C94EB050C94EB050C94EB050C948D1BA8
:100060000C94EB050C94EF1C0C941A1D0C947A1D47
:100070000C94EB050C94EB050C94EB050C94D71D3C
:100080000C94EB050C94901D0C94EB050C94EB0573
:100090000C94D71B0C94EB050C94EB050C94EB051E
:1000A0000C94EB050C94EB050C94EB05084AD73B3C
:1000B0003BCE016E84BCBFFDC12F3D6C74319ABD37
:1000C00056833DDA3D00C77F11BED9E4BB4C3E915B
:1000D0006BAAAABE000000803F05A84CCDB2D44E4A
:1000E000B93836A9020C50B9918688083CA6AAAA4C
:1000F0002ABE000000803F07634236B79BD8A71A8C
:1001000039685618AEBAAB558C1D3CB7CC5763BD99
:100110006DEDFD753EF6177231BF000000803F089F
:10012000000000BE922449123EABAAAA2ABECDCC42
:10013000CC4C3E00000080BEABAAAAAA3E00000044
:1001400000BF000000803F0000000000084178D39D
:10015000BB4387D1133D190E3CC3BD4282AD2B3E3C
:1001600068EC8276BED98FE1A93E4C80EFFFBE01DC
:10017000C4FF7F3F0000000000002D2D2D2D2D2DF0
:10018000202000003731322D3035202000B93731A2
:10019000322D3230202000643731322D3330202090
:1001A00000423735382D3530422000283735382D7C
:1001B0003130304200143735382D31353042000DA2
:1001C0003735382D32303042000A3735382D35304A
:1001D0005520003C3735382D313030550028373523
:1001E000382D31353055001B3735382D32303055EC
:1001F000001461637469762023257500412564002D
:100200002D2D0025733A202575204F686D0025732C
:100210003A202575204F686D0025733A20257520FA
:100220004F686D00474E44005663630044256400E8
:100230006175746F20002D2D006D616E2053573A4B
:100240002000442564002D2D0025736163746976B8
:100250002573003F3F204D56616C3A2578203F3F83
:100260000025642525002D2D2D2D2D2D202000006D
:100270003731322D3035202000B93731322D323030
:10028000202000643731322D3330202000423735B2
:10029000382D3530422000283735382D3130304266
:1002A00000143735382D31353042000D3735382DB3
:1002B00032303042000A3735382D35305520003C79
:1002C0003735382D3130305500283735382D313518
:1002D0003055001B3735382D32303055001425731A
:1002E00000302E25303275206D2F7300256C75255A
:1002F00073004D554925642000256C646D4100252F
:10030000756D56002573616374697600232564005A
:100310002074686F6D61734074686C732E6465003F
:10032000667265652052414D3A2575007C206578DE
:100330006974202F2073617665203C3E0020205890
:1003400053656E73202056312E37342E3100253000
:1003500032580020205853656E736F7220627920E6
:1003600054684C00636F6E666967206368616E67EE
:100370006564000010202020202020202020202044
:100380002020200001703A53656E736F7220636FF6
:100390006E66696700F1F03A5265736574205661C4
:1003A0006C7565732000E1B03A53657475702F4920
:1003B0006E666F2020200002F03A53656E736F72F4
:1003C00020416C74203C3E0003302E53656E732038
:1003D000416C74546F743C3E0004302E53656E7350
:1003E0002054656D7020203C3E0005302E53656E14
:1003F0007320566172696F203C3E0006202E4669CC
:100400006C74202020446561647A2E0012F03A5307
:10041000656E736F72204750532020200013302EDA
:1004200053656E7320506F732020203C3E001430C3
:100430002E53656E7320416C742020203C3E0015C5
:10044000302E53656E73205370656564203C3E000A
:1004500016302E53656E732044697374546F3C3E9E
:100460000017302E53656E73205472697020203C43
:100470003E0018202E53656E732053617473202044
:100480003C3E0022F03A53656E73205069746F74DD
:100490002020200023202E506F7274202020202046
:1004A000203C2D3E0032F03A53656E7320566F6C3F
:1004B00074616765200033302E46756E6374696F12
:1004C0006E20203C2D3E0034302E506F7274202060
:1004D000202020203C2D3E0035302E52657369735C
:1004E000746F7220203C2D3E0036202E52657369B9
:1004F00073746F7220203C2D3E0042F03A53656EBB
:1005000073204D554920746F74200043302E547968
:1005100070204143532020203C2D3E0044302E507B
:100520006F72742063757272203C2D3E0045302E30
:10053000636170612072657365743C2D3E004630C6
:100540002E506F727420766F6C74203C2D3E0047E5
:10055000302E5265736973746F7220203C2D3E00FB
:1005600048202E5265736973746F7220203C2D3EB3
:100570000052F03A536368616C7465722020203C2D
:100580003E0053302E506F72742053572020203C71
:100590002D3E00F2302E4361706163697479202032
:1005A000203C3E00F3302E5370656564206D617809
:1005B00020203C3E00F4302E4469737420746F7424
:1005C000616C203C3E00F5302E416C7420746F74D9
:1005D000616C20203C3E00F6202E7468617473200C
:1005E000616C6C2063796100E2302E53656E736F2D
:1005F00072204E622020203E00E3302E576174634B
:1006000068646F672020203C3E00E4302E41444364
:10061000205265665663633C2D3E00E5302E4D55F5
:10062000492063616C6962203C2D3E00E6302E66F5
:100630006163746F7279206465663C3E00E7302E1A
:1006400028632954682E4C65686D616E6E00E82041
:100650002E4465627567202020202020202000077E
:100660000605040100080A0B0C0D09000000002417
:100670000027002A002D003000000000002500287F
:10068000002B002E0031000000000023002600296E
:10069000002C002F000404040404030405020202D9
:1006A000020403020202020606060606060404020B
:1006B000020204040408020110408040102040801F
:1006C00040800802040180402010020110801020A8
:1006D0004040200000000200090F00000304010058
:1006E0000C000000000000000000000000000000FE
:1006F00000001E414C542E416C7469742E207265AA
:100700006C006D0000000001001F414C542E746FFE
:1007100074616C0000000000006B6D0000000402BA
:1007200020414C542E54656D700000000000000004
:10073000B043000000010123414C542E5661726900
:100740006F0000000000006D2F73000004022847B6
:1007500050532E536174656C6C697465730023008B
:100760000000000100294750532E4C6174697475D4
:100770006465000000200000000009002A47505373
:100780002E4C6F6E67697475646500002000000070
:100790000009002B4750532E416C746974756465D1
:1007A0000000006D0000000001002C4750532E5344
:1007B000706565640000000000006B6D2F6800012B
:1007C000002D4750532E5370656564206D61782E5F
:1007D000006B6D2F680001002E4750532E48656155
:1007E00064696E6700000000B00000000001002F87
:1007F0004750532E436F7572736520746F0000B0BD
:10080000000000000100304750532E4469737420EB
:10081000746F000000006D000000000100314750BF
:10082000532E44697374207472697000006D000067
:1008300000000400324750532E4469737420746FD3
:1008400074616C006B6D0000000402375069746FB6
:10085000742E5370656564000000006B6D2F680096
:1008600001003C566F6C746167652E31000000001A
:100870000000560000000001023D566F6C74616775
:10088000652E32000000000000560000000001024A
:100890003E566F6C746167652E33000000000000E7
:1008A000560000000001023F566F6C746167652EB0
:1008B0003400000000000056000000000102405615
:1008C0006F6C746167652E350000000000005600F3
:1008D000000000010241566F6C746167652E36009E
:1008E00000000000005600000000010242566F6C3C
:1008F000746167652E37000000000000560000009C
:1009000000010243566F6C746167652E3800000069
:100910000000005600000000010244566F6C746134
:1009200067652E390000000000005600000000013D
:100930000245566F6C746167652E3130000000000F
:10094000005600000000010246566F6C7461676536
:100950002E31310000000000560000000001024767
:10096000566F6C746167652E3132000000000056CE
:10097000000000000102484D5549312E4375727246
:10098000656E74000000410000000004024C4D55EB
:1009900049322E43757272656E740000004100008A
:1009A00000000402504D5549332E43757272656E36
:1009B0007400000041000000000402494D55493117
:1009C0002E566F6C746167650000005600000000D1
:1009D00001024D4D5549322E566F6C7461676500AA
:1009E000000056000000000102514D5549332E56BB
:1009F0006F6C746167650000005600000000010222
:100A00004A4D5549312E506F776572000000000045
:100A1000570000000004004E4D5549322E506F77AC
:100A20006572000000000057000000000400524DF5
:100A30005549332E506F7765720000000000570053
:100A400000000004004B4D5549312E436170616335
:100A500069747900006D4168000004004F4D5549EC
:100A6000322E436170616369747900006D416800E2
:100A7000000400534D5549332E436170616369741E
:100A80007900006D4168000004006453572D4569EA
:100A90006E67616E6731000000000000000000001A
:100AA000006553572D45696E67616E67320000001F
:100AB00000000000000000006653572D45696E6776
:100AC000616E673300000000000000000000006756
:100AD00053572D45696E67616E6734000000000052
:100AE0000000000000000000000000000000000006
:100AF00000000000000000000000000000585365E6
:100B00006E7300080B0002020200000904000001DD
:100B10000202000005240010010524010101042443
:100B200002060524060001070581031000400904A0
:100B30000100020A0000000705020240000007054C
:100B400083024000000403090412010002EF0201C5
:100B5000409A230E80000101020301416461667224
:100B600075697400497473794269747379203332FA
:100B700075342035562031364D487A00257325646A
:100B800025632000B41E11241FBECFEFDAE0DEBFC4
:100B9000CDBF11E0A0E0B1E0E4E6FBE702C00590C4
:100BA0000D92A63AB107D9F724E0A6EAB1E001C058
:100BB0001D92A935B207E1F715E0C3ECD5E004C0FA
:100BC0002197FE010E94953CC23CD107C9F70E94C3
:100BD000D51E0C94B03D0C9400002091B2033091CE
:100BE000B3032115310559F0E4E08E9FC0011124B3
:100BF000280F391FF901408351836283738308955D
:100C00002091A60381E0213208F040C08091820348
:100C10008111FCCF8091A50392E09093820391E033
:100C2000909381039FEF9093800310927F03209312
:100C30007E03A5E8B3E0EEE5F3E090E029132DC0D4
:100C400010925D0390915D03880F892B80935D0363
:100C500080915C03813029F510925C0380915D03E3
:100C60008093BB0085EC8093BC008091820382302E
:100C7000E1F3809180038F3FB1F080918003803257
:100C8000A1F080918003803391F084E0109284037E
:100C90001092A6031092830308953D9131939F5FB4
:100CA000CDCF85EEE0CF80E0F1CF82E0EFCF83E0E3
:100CB000EDCF90915A03911103C08FEF9FEF0895EC
:100CC0004FB7F89492E09093E9009091F200292FA9
:100CD00030E01216130614F421E030E0232B29F043
:100CE00084E6809359038091F100992339F0209193
:100CF000F200211103C02BE62093E8004FBF992397
:100D0000E1F290E008952FB7F89483E08093E90032
:100D10009091E800892F807295FF04C09091F200B5
:100D200080E4891B2FBF08958091510381110DC06C
:100D300082E080934D0384E080934E031092500331
:100D400010924F0381E0809351038DE493E0089566
:100D5000CF93DF931F92CDB7DEB76983DC01ED91AE
:100D6000FC910280F381E02D41E050E0BE016F5F15
:100D70007F4F09950F90DF91CF91089583E0809385
:100D8000E9008091F200882319F08AE38093E8005B
:100D900008950E94830690E00895FC01848595855E
:100DA00097FD05C02FEF3FEF3587248708950C94FA
:100DB0005906CF93DF93EC018C859D8597FF04C086
:100DC0000E9459069D878C878C859D85DF91CF91E8
:100DD0000895FC018485958597FD0BC09FB7F89415
:100DE00082E08093E9008091F2009FBF90E001963D
:100DF00008959FB7F89482E08093E9008091F20013
:100E00009FBF90E00895409147035091480320917F
:100E100045033091460342175307B4F49091E8001C
:100E20009570E1F39091E80092FD19C08093F10074
:100E3000809147039091480301968F739927892BDE
:100E400019F48EEF8093E800809147039091480356
:100E50000196909348038093470381E0089580E0D2
:100E60000895DF92EF92FF920F931F93CF93DF933A
:100E7000D82E8A01EB017B01E40EF51ECE15DF05AD
:100E800059F0D7FE12C0FE0184910E9403072196FB
:100E90008111F4CF0FEF1FEFC801DF91CF911F91A8
:100EA0000F91FF90EF90DF9008958881EECF0F9320
:100EB0001F93CF93DF931F92CDB7DEB782E0898374
:100EC00042E450E063E07BE080E80E9431070E944A
:100ED0009406DC0112960D911C910115110589F003
:100EE000D801ED91FC910280F381E02DBE016F5F8E
:100EF0007F4FC801099597FD04C0F8010085118551
:100F0000ECCF89810F90DF91CF911F910F910895C0
:100F100081508F3008F047C0E82FF0E0EE56F84FD0
:100F20000C94953CAF07B307A107A707AB07D307FE
:100F3000D307D307B607BC07C007C407CA07D30740
:100F4000CE07809180008F778093800008958091F4
:100F500080008F7DF9CF80918000877FF5CF84B5A9
:100F60008F7784BD089584B58F7DFBCF80919000ED
:100F70008F77809390000895809190008F7DF9CFB6
:100F800080919000877FF5CF8091C0008F7780930C
:100F9000C00008958091C0008F7DF9CF8091C2007C
:100FA000877F8093C2000895CF93DF93282F30E08E
:100FB000F901ED52F94F8491F901EC54F94FD491B4
:100FC000F901EB56F94FC491CC23A1F081110E9495
:100FD0008807EC2FF0E0EE0FFF1FE957F94FA591BE
:100FE000B491EC91ED2381E090E009F480E0DF9191
:100FF000CF91089580E090E0FACF1F93CF93DF93D5
:10100000282F30E0F901ED52F94F8491F901EC54A9
:10101000F94FD491F901EB56F94FC491CC23A9F0C3
:10102000162F81110E948807EC2FF0E0EE0FFF1FB2
:10103000E758F94FA591B4918FB7F894EC9111113D
:1010400008C0D095DE23DC938FBFDF91CF911F9135
:101050000895DE2BF8CFCF93DF9390E0FC01EC54A2
:10106000F94F24918B56994FFC0184918823D1F03C
:1010700090E0880F991FFC01E559F94FA591B491B3
:10108000FC01E758F94FC591D491623071F49FB7D4
:10109000F8943C91822F809583238C93E8812E2BAA
:1010A00028839FBFDF91CF9108958FB7F894EC917B
:1010B0002E2B2C938FBFF6CF823108F08251E82F70
:1010C000F0E0E15AF94FE49190917B008E2F880F68
:1010D000880F80729F7D892B80937B00E770E0648E
:1010E000E0937C0080917A00806480937A00809104
:1010F0007A0086FDFCCF8091780090917900089568
:101100003FB7F89480911E0290911F02A091200297
:10111000B091210226B5A89B05C02F3F19F001967A
:10112000A11DB11D3FBFBA2FA92F982F8827BC0141
:10113000CD01620F711D811D911D42E0660F771F69
:10114000881F991F4A95D1F708958F929F92AF9269
:10115000BF92CF92DF92EF92FF924B015C010E940F
:1011600080086B017C010E9480086C197D098E0942
:101170009F09683E734081059105A8F321E0821A1A
:101180009108A108B10888EEC80E83E0D81EE11CC2
:10119000F11C81149104A104B10429F7FF90EF9090
:1011A000DF90CF90BF90AF909F908F9008958F92D7
:1011B0009F92AF92BF92CF92DF92EF92FF920F93E6
:1011C0001F93CF93DF936C017B018A0180910B0108
:1011D000882309F45BC080915A03882309F456C020
:1011E00080914C0380FF05C08091E0008260809375
:1011F000E000E801B12C8AEFA82E93E0892E2AE3C3
:10120000922E209711F4BB20D9F10E948306811100
:101210000AC0AA94AA20D1F161E070E080E090E0D9
:101220000E94A508EECF8C171D0611F00CF08C2F34
:101230009FB7F8948092E9002091E80025FD02C054
:101240009FBFDFCF282F30E0C21BD30BF7018150A7
:1012500020F041914093F100FACFE20EF31EBB2043
:1012600021F09092E800B12CEBCF8091E80085FD51
:10127000E7CF9092E800BB24B394209709F3F3CF13
:1012800084E680934B03101611063CF081E090E059
:10129000F6019383828310E000E0C801DF91CF91D3
:1012A0001F910F91FF90EF90DF90CF90BF90AF9084
:1012B0009F908F9008952FB7F89460911A027091C3
:1012C0001B0280911C0290911D022FBF089585ED95
:1012D0008093BC008091BC0084FDFCCF10928203FF
:1012E0000895613298F420918203243089F4609348
:1012F000F601282FA6EDB1E0FC018E2F821B861788
:1013000010F080E0089581918D93F7CF81E00895EA
:1013100082E008950895E091230280912202E81767
:1013200030F4F0E0EA54FE4F808190E008958FEFB2
:101330009FEF089590912302809122022FEF3FEFBB
:10134000981748F4E92FF0E0EA54FE4F208130E08E
:101350009F5F90932302C90108958091220290918A
:101360002302891B990B0895CF92DF92EF92FF928F
:101370000F931F93CF93DF937C01CB018A012091C0
:101380008303222389F0EB016B01C40ED51ECC151B
:10139000DD0569F06991D701ED91FC910190F08133
:1013A000E02DC7010995F3CF642F0E947109C80190
:1013B000DF91CF911F910F91FF90EF90DF90CF9031
:1013C0000895CF93DF931F92CDB7DEB76983209145
:1013D00083032223F9F02091A603203258F021E064
:1013E00030E0FC013383228390E080E00F90DF91B6
:1013F000CF91089580918403E82FF0E0EB57FC4FE4
:10140000998190838F5F809384038093A60381E00A
:1014100090E0ECCF61E0CE0101960E947109F7CF18
:1014200090E080E00895FB01803E51F481E08093DC
:10143000AF0180819181480F591F518340830895E6
:10144000803761F4808191818417950738F021E01D
:101450002093AF01841B950B918380830895803E78
:1014600061F481E0860F841768F4222371F08617F7
:1014700061F091E09093AF010895803729F46623DD
:1014800019F0862F8150F1CF862F0895CF93DF93E7
:10149000EC018A859B85AC85BD858E839F83A8875B
:1014A000B9870E945B096A837B838C839D8381E07B
:1014B00089838883DF91CF910895CF92DF92EF9255
:1014C000FF92CF93DF93EC0119826B857C858D852C
:1014D0009E850E94DB3828E23BE64EE65EE40E94F1
:1014E00033386B017C0169857A8590E080E00E9449
:1014F000DB389B01AC01C701B6010E944B372F8539
:1015000021119058DF91CF91FF90EF90DF90CF9015
:101510000895CF92DF92EF92FF92CF93DF93EC0189
:1015200019826C817D818E819F810E94DB3828E247
:101530003BE64EE65EE40E9433386B017C016A8133
:101540007B8190E080E00E94DB389B01AC01C70109
:10155000B6010E944B37288521119058DF91CF9119
:10156000FF90EF90DF90CF900895CF92DF92EF92AF
:10157000FF920F931F93CF93DF93EC018881882311
:1015800039F10E945C088C0169817A8190E080E0E9
:101590000E94DB3820E030E040E45FE30E94343A10
:1015A0006B017C01B801110F880B990B0E94DD388B
:1015B00020E030E040E85EE30E94343A9B01AC0159
:1015C000C701B6010E944B370E94AC387A83698309
:1015D00089819A81DF91CF911F910F91FF90EF90B8
:1015E000DF90CF9008958F929F92AF92BF92CF924B
:1015F000DF92EF92FF920F931F93CF93DF93EC0153
:10160000162F888990E082579D4FFC01ED57FF4FC0
:1016100000818A579F4FFC01608170E090E080E07C
:101620000E94DD386B017C016091DD027091DE0269
:1016300090E080E00E94DB38083008F0CFC020E066
:1016400030E040E05FE30E94343A20E030E04AEFCF
:1016500052E40E944A37A70196010E944B376B0162
:101660007C01888599850E94B50A2AE0029FF001D5
:101670001124ED57FE4F0491BC0190E080E00E94E0
:10168000DB3820918F02309190024091910250916D
:1016900092020E94343AA70196010E944A3720E044
:1016A00030E04AE754E40E94343A6B017C01602F39
:1016B00070E090E080E00E94DD389B01AC01C70142
:1016C000B6010E9433386B017C0120E030E0A901B3
:1016D0000E94293887FF05C0111103C0C12CD12CED
:1016E00076010E945B09088D198D2A8D3B8D601B48
:1016F000710B820B930B688F798F8A8F9B8F088970
:10170000E4E00E9F800111240A541D4F0E94DB3833
:10171000A70196010E94343A20E03AEB4BE55AE4E7
:101720000E943338F80120813181428153810E9427
:101730004B37F80160837183828393830E945B0936
:10174000688F798F8A8F9B8F088910E0065F1F4F03
:10175000F801EE0FFF1FEE0FFF1FE257FD4F8080D5
:101760009180A280B3806E897F8990E080E00E94A2
:10177000DB389B01AC01C501B4010E94F339181696
:101780006CF4C501B4010E94AC386F5F7F4F7F8B52
:101790006E8B80918E02816080938E02000F111FEC
:1017A000000F111FF801E257FD4F608171818281A6
:1017B00093810E94AC387F836E83C701B6010E947B
:1017C000A538DF91CF911F910F91FF90EF90DF909F
:1017D000CF90BF90AF909F908F9008952EEA37E4FE
:1017E00045E051E40E94333830CFCF93DF93EC01D2
:1017F00081E08093830387E78093A503109284039D
:101800001092A60389E494E00E94E1090E94000678
:1018100091E0811101C090E09883DF91CF9108950C
:10182000CF92DF92EF92FF92CF93C42F0E94F50BDD
:10183000809182038111FCCF9C2F81E080938203F1
:10184000809381032FEF2093800310927F032C0F4E
:1018500020937E0380935D0380915D038E6E809361
:101860005D0380915C038130B1F510925C0380913F
:101870005D038093BB0085EC8093BC008091820364
:101880008130E1F380917F038C1710F490917F03F6
:10189000EEE5F3E0A6EBB1E0C0E0C9131EC0109284
:1018A0002302C093220260E070E0CB01209123026A
:1018B000C217B9F0CC24D62EE72EF82E89E494E096
:1018C0000E949A09BC01990F880B990B6C297D29FC
:1018D0008E299F29EBCF85EECFCF81918D93CF5F5E
:1018E000DCCFCF91FF90EF90DF90CF900895CF9312
:1018F000DF93F894EC01CA57DF4F28812034E0F4DD
:1019000070E030E020E0442311F020E031E0DC0121
:10191000AE57BF4F622B732BED91FC9111977183E2
:101920006083329628812F5F2883EA17FB0710F027
:10193000FC013296ED93FC93FC01E757FF4F808149
:10194000811108C081E080838091C9008F76886210
:101950008093C9007894DF91CF910895CF93DF935E
:10196000DC01A857BF4F2C91222351F0FC01E9570D
:10197000FF4F8081EB018883F89410821C92789449
:10198000822FDF91CF910895CF93DF93EC011092D6
:10199000C8008CE08093C90086E38093CA0010924F
:1019A000CD0086E68093CC0062E080E00E942B08A8
:1019B00062E081E00E942B08CE010296FE01EE5704
:1019C000FF4F918380833296918380833296108279
:1019D00033961082D093AB01C093AA01DF91CF91CF
:1019E000089508954F925F926F927F92AF92BF9247
:1019F000CF92DF92EF92FF920F931F93CF93DF93DB
:101A000000D000D0CDB7DEB7082FA62E69017A012D
:101A1000AE014F5F5F4FC701B9010E94003A2B0131
:101A20003C0169817A818B819C819F770E94AC38CF
:101A3000B62E172F2AE939E949E15FE3C301B20164
:101A40000E94343A20E030E543EC57E40E94343AF7
:101A50009F770E94AC383B01117070E0A11070E2DA
:101A6000172B20E030E0A901C701B6010E942938F8
:101A700070E087FD70E4712BA3016B2D802F0F9018
:101A80000F900F900F90DF91CF911F910F91FF90CA
:101A9000EF90DF90CF90BF90AF907F906F905F906E
:101AA0004F900C94ED05EF92FF920F931F93CF93FD
:101AB000DF93CDB7DEB767970FB6F894DEBF0FBEE2
:101AC000CDBF9B0143E0359527954A95E1F7E0911D
:101AD000A703F091A803E20FF31F208130E0AB01D0
:101AE0004770552702C0359527954A95E2F7217032
:101AF0003327DC0117962C93232B09F468C07B0154
:101B00008C0127E1269FC001279F900D1124609131
:101B1000B0037091B103680F791F47E150E0CE0127
:101B200001960E9437348981F8018283A801485FB9
:101B30005F4F9E012E5F3F4FDA0180E0F9019191E6
:101B40009F01992329F0833119F08F5F9D93F6CF80
:101B5000D8015C968C93DE015196FA01E80FF11DD5
:101B600090E02D91222339F0382F390F333118F4BA
:101B70009F5F2193F6CFD8015D969C931082EE0C67
:101B8000FF1CEE0CFF1C6091B2037091B303E60ED4
:101B9000F71EF70180819181A281B381F8018383CF
:101BA0009483A583B6838F89813021F08230E1F060
:101BB000178E02C080E2878F8E89F801868F86306B
:101BC000B0F4843010F58823B9F08130D1F06796F5
:101BD0000FB6F894DEBF0FBECDBFDF91CF911F913E
:101BE0000F91FF90EF90089580E4878FE5CF8850A4
:101BF000823068F785E006C082E0D80190968C9329
:101C0000E6CF83E0F80180A3E2CF84E0F6CF5F92D5
:101C10006F927F928F929F92AF92BF92CF92DF92FC
:101C2000EF92FF920F931F93CF93DF93CDB7DEB761
:101C3000162FF72EB42E552E3901402F2E2D80361B
:101C400031F490915B0331E0932790935B03909183
:101C50005B03911132C0F30160810E942F0AF301EE
:101C6000808380915B038823A9F18EE31F928F9379
:101C7000F301808190E001969F938F935F92BF92D2
:101C80008CE79BE09F938F93FF921F930E945C349D
:101C90000FB6F894DEBF0FBECDBFDF91CF911F917D
:101CA0000F91FF90EF90DF90CF90BF90AF909F90FB
:101CB0008F907F906F905F900895FFEF8F169F0633
:101CC00081F2282D21704A2DF60160810E942F0A91
:101CD000F601C6CF8CE3CACF211126E030E04617CB
:101CE000A0F0E62FE695E695E695F0E0EC52FD4F84
:101CF000E081F0E0562F577002C0F595E7955A95B0
:101D0000E2F7E0FD3F5F6F5FEACF1F923F9330E065
:101D10002E503E4F3F932F939F938F930E945C349E
:101D20000F900F900F900F900F900F9008954F927B
:101D30005F926F927F928F929F92AF92BF92CF925B
:101D4000DF92EF92FF920F931F93CF93DF93CDB764
:101D5000DEB760970FB6F894DEBF0FBECDBF6983C4
:101D60007A838B839C83CA01B9012701A60195015F
:101D70000E944A3725E33AEF4EE85CE30E94343A8A
:101D80006B017C010E94F13A6D877E878F87988B6B
:101D9000C701B6010E942E386D837E838F8398879A
:101DA00025E33AEF4EE85CE369817A818B819C817F
:101DB0000E94343A4B015C0125E33AEF4EE85CE3C4
:101DC000C801B2010E94343A2B013C01C501B401A3
:101DD0000E94F13A69837A838B839C83C501B401A5
:101DE0000E942E384B015C01C301B2010E94F13AFE
:101DF00069877A878B879C87C301B2010E942E383E
:101E00006B017C0129853A854B855C85C501B40150
:101E10000E94343A2B013C01A701960169817A8125
:101E20008B819C810E94343A2D813E814F8158855F
:101E30000E94343A9B01AC01C301B2010E944A37AF
:101E40009B01AC010E94343A2B013C01A701960191
:101E50006D857E858F8598890E94343A9B01AC01FF
:101E60000E94343AA30192010E944B370E94FF3A2C
:101E70002B013C01A7019601C501B4010E94343A2F
:101E80002D813E814F8158850E94343A4B015C017F
:101E900029853A854B855C8569817A818B819C8116
:101EA0000E94343A9B01AC01C501B4010E944B373A
:101EB0009B01AC01C301B2010E94CA3726E73BE790
:101EC00042EC5AE40E94343A60960FB6F894DEBFB2
:101ED0000FBECDBFDF91CF911F910F91FF90EF907B
:101EE000DF90CF90BF90AF909F908F907F906F903A
:101EF0005F904F900895FF920F931F93CF93DF93BE
:101F00008C01EB01F8808DE2F81201C02196CE0120
:101F10000E9410349B01AC01A4E6B0E00E949B3CFF
:101F2000AB01BC01FE012991822F022E000C990BFE
:101F3000C0970A97B8F32E3231F58181082E000C34
:101F4000990BC0978A309105F0F4AAE0A89F900100
:101F5000A99F300D1124C901330FAA0BBB0B480FE9
:101F6000591F6A1F7B1F8281082E000C990BC09796
:101F70008A30910540F4092E000CAA0BBB0B480FC8
:101F8000591F6A1F7B1FEDE2FE1207C07095609516
:101F9000509541955F4F6F4F7F4FF80142875387B0
:101FA00064877587DF91CF911F910F91FF900895FE
:101FB0002F923F924F925F926F927F928F929F9259
:101FC000AF92BF92CF92DF92EF92FF920F931F9347
:101FD000CF93DF93D82FC92F8B010E94103424E6B2
:101FE00030E040E050E00E94543C49019B01AC01CC
:101FF00060E876E988E990E00E94303C6B017C0162
:10200000F80191828082ED2FFC2F2191822F022EE8
:10201000000C990BC0970A97C0F32E3239F51F01B7
:1020200080E8882E86E9982E88E9A82EB12C9AE0BF
:10203000492E512C612C712CF101C1911F010C2EE4
:10204000000CDD0BE097CA30D10580F4C501B40166
:10205000A30192010E94543C49015A01DE010E94F1
:10206000A63CC60ED71EE81EF91EE6CFA5E0B0E0DE
:10207000A70196010E949B3C6F5F7F4F8F4F9F4F40
:1020800023E030E040E050E00E94543CF80122831D
:102090003383448355831682DF91CF911F910F9133
:1020A000FF90EF90DF90CF90BF90AF909F908F9078
:1020B0007F906F905F904F903F902F900895EF9298
:1020C000FF920F93CF93DF937C01EA016111E90145
:1020D0000039D1F58091AD0191E089278093AD0160
:1020E0006623D9F168E272E0C7010E94403483E0C0
:1020F000E80EF11C8091AD01882391F145E050E09C
:10210000BE01802F0E94130A89818F9388818F934B
:102110008DE591E09F938F9389E192E09F938F9358
:10212000FF92EF920E945C341092AC018DB79EB783
:1021300008960FB6F8949EBF0FBE8DBFDF91CF916A
:102140000F91FF90EF900895003651F68091AC0109
:1021500091E089278093AC01C3CF64E272E0C4CFE1
:102160008091AC01882309F148EE53E0BE01802F35
:102170000E94130A89818F9388818F9381E691E071
:102180009F938F938EE092E09F938F93FF92EF92B5
:102190000E945C341092AD018DB79EB708960FB6C1
:1021A000F8949EBF0FBE8DBFC9CF44E650E0BE017C
:1021B000802F0E94130A89818F9388818F938FE7E4
:1021C00091E09F938F9383E092E09F938F93FF9290
:1021D000EF920E945C348DB79EB708960FB6F894C4
:1021E0009EBF0FBE8DBFAACFCF92DF92EF92FF921C
:1021F0000F931F93CF93DF93CDB7DEB72D970FB615
:10220000F894DEBF0FBECDBFD82EC92E162F7A018F
:10221000822F9DE0E2E1F1E0DE01119601900D9246
:102220009A95E1F7FA019081FE01319660E02191E3
:10223000921719F06F5F6D30D1F721E04DE00E94E9
:102240002F0A21E030E02C0F3D1F280F311DF9012E
:102250008081F7018083012F17FF02C007E0010F83
:10226000059505950595202F000F330B177817FF5F
:1022700003C01150186F1F5F41E050E07A0101C0A8
:10228000EE0C1A95EAF7890102571D4F81111DC006
:1022900060E072E08D2D9C2D0E944034F801EA5BD5
:1022A000FF4FE0948081E822E08280E02D960FB617
:1022B000F894DEBF0FBECDBFDF91CF911F910F917C
:1022C000FF90EF90DF90CF900895082E000C990BAF
:1022D00042979F938F938CEF91E09F938F93CF9230
:1022E000DF920E945C34F801EA5BFF4F8081E82AAC
:1022F000E0820F900F900F900F900F900F9081E061
:10230000D5CF80919602909197028832964169F0DC
:10231000E8E9F2E08AE3DF011D928A95E9F788E2B5
:1023200096E190939702809396028091D2029091C9
:10233000D30284309841E9F0E4EDF2E089E6DF0170
:102340001D928A95E9F784E098E19093D3028093F7
:10235000D20288E893E19093DE028093DD0280E56B
:102360008093DF028DE7809314038093150380939D
:1023700016036091DD027091DE0290E080E00E9421
:10238000DB3820E030EC4FE754E40E9433386093B0
:102390008F0270939002809391029093920208951D
:1023A000DF92EF92FF920F931F93CF93DF93F82E5C
:1023B0009CE3E92E611102C087EAE82EF1100E9429
:1023C00081110EE812E0D0E0C0E0FF20D9F0F80162
:1023D000D084CE010E94FD36D81621F06D2DCE019D
:1023E0000E94053721960F5F1F4FCE1570F3F11035
:1023F0000FC0DF91CF911F910F91FF90EF90DF9071
:102400000C948111CE010E94FD36F8018087EACF3D
:10241000DF91CF911F910F91FF90EF90DF90089582
:102420002F923F924F925F926F927F928F929F92E4
:10243000AF92BF92CF92DF92EF92FF920F931F93D2
:10244000CF93DF93CDB7DEB769970FB6F894DEBFB1
:102450000FBECDBF882309F46AC08FEF898F898DA5
:10246000803F41F0982F9F7029F49091B501891712
:1024700009F46DC08093B501882309F468C08FEF1B
:10248000809347026091B401B1E16B9FB0011124C8
:102490006D587C4F42E050E0CE0147960E943734A1
:1024A000898D803B09F4A4C008F06AC0803709F424
:1024B00083C0803919F0803609F049C08091B2019B
:1024C0008F708093B201E0E18E9FC00111240091D2
:1024D000B301802B2DE2F22E082F10E031E1E32E24
:1024E0008F89988D8017110609F48EC08091B401F0
:1024F0008F5F8C3208F085C08093B4016091B40185
:102500006E9DB00111246D587C4F42E050E0CE0129
:1025100047960E943734FA94F110E2CF8091B101CE
:102520008093B2018091B0018093B30110C080917B
:10253000B7039091B803DC01ED91FC910480F58123
:10254000E02DBE01675E7F4F0995811188CF6996A6
:102550000FB6F894DEBF0FBECDBFDF91CF911F91B4
:102560000F91FF90EF90DF90CF90BF90AF909F9032
:102570008F907F906F905F904F903F902F90089535
:10258000803E29F18F3F09F499CF803D01F7888D76
:1025900085FF94CF8091B30181508093B30188234C
:1025A00041F0813009F08ACF8091B2018E3008F07D
:1025B00085CF1092B20182CF888D87FF7FCF809127
:1025C000B2019091B301913059F48F5F0AC0888DA8
:1025D00086FF74CF8091B2019091B301913021F4C4
:1025E00081508093B2016ACF853008F067CFEDCF7C
:1025F000888D84FF63CF8091B3018F5F8093B30197
:102600005DCF1092B4017ACF2091B2012093B10135
:102610002091B3012093B0019E012F5F3F4F3901FC
:102620008115904109F04FC08091AF0164E673E0DD
:10263000811102C063E573E0C3010E9440341301BD
:10264000E7EAF3E09E012F5E3F4F230180E040E286
:10265000D2019D912D01992309F454C0811152C0DA
:1026600092AB31962415350599F740E150E060E2D0
:1026700070E0C3010E94A03D6F89788D6534B0E39E
:102680007B0709F447C408F06BC16530F0E37F07AE
:1026900009F42EC308F0DDC0663330E2730709F495
:1026A00082C308F046C0663050E2750709F425C3BE
:1026B00060F5611590E1790709F477C27F936F9314
:1026C00083E592E057C01F930F938EE493E09F93AE
:1026D0008F937F926F920E945C346091B40141E1CC
:1026E000649FB00111246B587C4F4FE050E0CE0145
:1026F00003960E9437340F900F900F900F900F9019
:102700000F909DCF42AB81E0ACCF6831A0E27A0759
:1027100009F4B7C46332B0E27B0781F6298D46E243
:1027200053E06FE0C3010E94F41081E08093AF0199
:102730006AC2663FE0E27E0709F465C200F56834CC
:1027400020E2720709F461C4683E30E2730709F0C1
:10275000B5CF9E012E5E3F4F809155049091560457
:10276000009711F489E594E0281B390B3F932F93D0
:1027700080E293E09F938F937F926F9214C46330B3
:1027800040E3740709F41BC510E082E0643050E3B5
:10279000750709F093CF982FE92EE594E594E59419
:1027A0000E2C000CFF08082F0770998D903681F4CD
:1027B000F701EC52FD4F21E030E0002E01C0220F66
:1027C0000A94EAF790819227908391E09093AF0169
:1027D00087FD22C0F701EC52FD4F808190E0002E72
:1027E00002C0959587950A94E2F780FFE2C48FE7CF
:1027F00091E02FE731E03F932F939F938F9389E4EC
:1028000092E09F938F937F926F920E945C340FB6F9
:10281000F894DEBF0FBECDBF809147028F3F51F0CD
:1028200080914D0290914E026AE070E00E94403C1F
:102830008063888BF701E258FD4F868190E002C0EB
:10284000959587950A95E2F780FFFDC389E48F8708
:10285000FAC3673180E3780709F407C498F5643157
:10286000A0E37A0709F49EC1B8F46331E0E37E0780
:1028700009F024CF898D803661F48091D40290E4F0
:1028800089278093D4028091D50294E08927809390
:10289000D50210E085E07FCF6531F0E37F0709F4D2
:1028A000D8C3663120E3720709F008CF898D8036DE
:1028B00031F48091D50298E089278093D50210E009
:1028C0008CE069CF653330E3730709F46CC270F5AF
:1028D000633350E3750709F44AC2643380E3780731
:1028E00009F0ECCE88248A94982CA12CD12CC12CF0
:1028F000E12C0CE02EEA31E040E851E0B301898D93
:102900000E94070E20915B03211101C0198E609176
:10291000AE01462F50E0435D5C4F605F298D860D10
:10292000971D0E94F4101092AD016DC1633490E3C5
:10293000790709F462C26434A0E37A0709F0BECED5
:102940006091AE01462F50E0FA01EF5EFC4F8081AE
:102950008111A4C28091B30181508093B301C0C0A2
:10296000633FB0E37B0709F41AC108F0BFC0633EC0
:10297000F0E37F0709F466C120F5673430E373079D
:1029800009F443C308F415C3633550E3750709F42C
:102990007FC3623E80E3780709F090CE898D803E48
:1029A00041F48091DA028E5F8093DA0281E08093B5
:1029B000AF018091DA0286951F928F938CE093E0AD
:1029C000D9CE663E90E3790709F468C108F044C0A7
:1029D000643EB0E37B0709F451C1653EE0E37E0746
:1029E00009F06CCEC090AE01D12CD601AC5EBC4FCC
:1029F0006D0188248394912C8AEFA82EE12C03E0AA
:102A00002EEA31E049E751E0B301898D0E94070EBB
:102A10008C01E091AE01F0E0EE0FFF1FE25AFD4F96
:102A200080819181009709F4EEC061E00E94F30A71
:102A30009F938F937F936F9389EF92E09F938F93F0
:102A4000060D171D1F930F930E945C340FB6F89468
:102A5000DEBF0FBECDBFD7C0673EF0E37F0709F4EE
:102A6000CDC0623F20E3720709F028CE20E043E0AA
:102A70006091AE01898D0E942F0A8093AE0190E093
:102A800001969F938F9382EF92E09F938F937F9213
:102A90006F920E945C340091AE01F4E00F9F8001C0
:102AA00011240A541D4FD8016D917D918D919C91F7
:102AB0000E94AC380F900F900F900F900F900F90D6
:102AC00025E048E651E0398D303609F0F5C0F801CF
:102AD000108211821282138260E081E00E94D01184
:102AE00080918E02826080938E028DC0623130EFC1
:102AF000730709F499C260F5613050E7750709F46E
:102B000082C098F4643F90E3790709F4D2C002EBE5
:102B100012E0653FA0E37A0709F0D0CD60E070E0F5
:102B2000CB0120E04FE751E0CECF613EB0EB7B0719
:102B300031F16230E0EF7E0709F0C0CDE091430350
:102B4000F091440310E0309709F0108180E023CE2B
:102B50006234F0EF7F0709F438C1A0F4623230EF3D
:102B6000730709F400C1623340EF740709F0A6CD82
:102B700020E04BE160E1CE0104960E946C0E1092C1
:102B80005B030AC0623550EF750709F47DC2613FEF
:102B900080EF780709F092CD1092AE0134C00EEAB2
:102BA00012E0BCCF10E087E0F6CD6DE373E0C30127
:102BB0000E9440348091DA02982F9E7F19F086950A
:102BC000805D88878091AF018823E9F06CE273E033
:102BD000C3010E944034898D803629F460E081E091
:102BE0000E94D01102C0803971F464E670E080E088
:102BF00090E00E94A5080C94000005C060E173E01D
:102C0000C3010E944034F30180E29191911103C00D
:102C1000DF0111978C934E165F06B9F749EE53E02A
:102C200080E020E2D1019D911D01DA01992309F490
:102C3000C3C28111C1C29C934F5F5F4FE215F30580
:102C400089F785CC898D803659F49091DA02892FE5
:102C50008E7F90FF81608093DA0281E08093AF01E4
:102C60008091DA0280FF07C08FE791E09F938F93F6
:102C700084E093E07FCD85E691E0F8CF45E050E039
:102C80006DED72E0898D0E94130A8091DE028F93B0
:102C90008091DD028F938FEF92E06CCD898D80362D
:102CA00009F0B1CF8FEF9FEF9093D3028093D202C0
:102CB00095CF0AEA12E032CF6115710581059105C1
:102CC00029F4D8016D917D918D919C915F934F93E3
:102CD0009F938F937F936F938CEE92E09F938F934C
:102CE000260D372D311D3F932F930E945C34AECEBD
:102CF00010925B0310E083E04ECD8091DF028150A3
:102D00008093DF0288248394912CB4E6AB2E10EEDE
:102D1000C12E12E0D12EEE24E39403E62FED32E033
:102D20004DE751E0BE016C5F7F4F898D0E94070E19
:102D30002091E0021F922F9321EE32E03F932F93D8
:102D40000396860D971D9F938F930E945C3480910C
:102D5000DF028F5F8093DF020F900F900F900F9034
:102D60000F900F9050CF198E10E08FE014CD898D09
:102D7000803659F49091DB02892F8E7F90FF81601D
:102D80008093DB0281E08093AF018091DB0280FDC4
:102D900007C08CE691E09F938F938EED92E0EACC92
:102DA00084E791E0F8CF4091AE0150E0440F551F09
:102DB0009A012F513D4F47505D4F655370436170ED
:102DC000098DC3010E945F101ECF20E04EE16CE12F
:102DD000CE0104960E946C0EE4E0F0E0EC0FFD1FC3
:102DE000E80FF91F2FE22083049621E047E26CE10F
:102DF000860D971D0E946C0ECFCE88248A94982C45
:102E0000A12CD12CC12CE12C03E02EEA31E049E7C2
:102E100051E0B301898D0E94070E8C0180915B0304
:102E2000811101C0198EE090AE01F12C97012F5E47
:102E30003C4F790121E04CE0D7016C91898D0E94D3
:102E40002F0AF7018083E091AE01F0E0EF5EFC4FC6
:102E50008081FAE08F9FC00111248A599D4F9F9372
:102E60008F93060D171D1F930F930E945C34909152
:102E7000AE01E92FF0E0EF5EFC4F0F900F900F9046
:102E80000F9080818111BFCE945E892F80688F3F23
:102E900009F4B9CE9F77198E10E07ECC495D5C4F66
:102EA000645E298DC3010E94F4109091AE018823C5
:102EB000B9F0892F90E08596FC0143E0F595E79500
:102EC0004A95E1F7EC52FD4F8770992721E030E0F9
:102ED00001C0220F8A95EAF78081822B808393CEEE
:102EE000892F90E08596FC0153E0F595E7955A957A
:102EF000E1F7EC52FD4F8770992721E030E0A901FE
:102F000002C0440F551F8A95E2F7CA01809590814F
:102F10008923E4CF0091AE0110E002571D4FF80164
:102F2000E757FF4F21E047E06081898D0E942F0A1B
:102F3000F82E51E060E372E0C3015F15B8F169E378
:102F400072E00E944034CE01099666E372E0FF20F1
:102F500069F11F9227E02F932CE232E03F932F93E9
:102F60009F938F930E945C340F900F900F900F905F
:102F70000F900F90F801E757FF4FF082E091AE01FC
:102F8000F0E0E95EFC4F8081833008F43CCE825053
:102F9000990B9F938F9381E692E09F938F93CE013D
:102FA00004969F938F930E945C34D6CE0E94403447
:102FB000E1CF1092AD016091AE01462F50E0465D29
:102FC0005C4F615E298DC3010E94F4109091AE01A7
:102FD000882321F0892F90E082966ECF892F90E090
:102FE0008296FC0133E0F595E7953A95E1F7EC52CE
:102FF000FD4F8770992721E030E0D90102C0AA0F68
:10300000BB1F8A95E2F7CD0181CF4091AE0150E020
:103010004A5B5F4F440F551F9A0122573D4F4C5654
:103020005D4F67547043CBCE20E04EE064E0CE01AC
:1030300004960E946C0EE0914103F0914203309798
:1030400009F4E1CD1081112309F4DDCD86E4888BEC
:10305000DACD898D803631F48091D50292E08927CE
:103060008093D50210E088E096CB898D803631F4CC
:103070008091D50290E489278093D50210E08DE0FD
:103080008ACB10E084E087CB20E04BE268E273CD8E
:1030900088248A94982CA12CD12CC12CE12C04E0FA
:1030A0002EEA31E045E851E0B301898D0E94070E18
:1030B0007C0180915B03811101C0198E598D909123
:1030C000AE01092F10E088E2B82EB90EE60CF71C0D
:1030D00095E0EFE1F1E0DE01529601900D929A95B4
:1030E000E1F70F551D4FF801E856FF4F2081022EE2
:1030F000000C330BFE01729660E06F018191821724
:10310000130619F06F5F6530C9F721E045E0852FA0
:103110000E942F0A8C0D9D2D911DFC019081F801BC
:10312000E856FF4F90830B2DB7FE02C007E00B0D52
:10313000059505950595002E000C110B8B2D8778B4
:1031400087FF03C08150886F8F5F21E030E0690105
:1031500001C0CC0C8A95EAF702571D4F91110EC0A1
:1031600066E472E0C7010E944034F801EA5BFF4F59
:103170008C2D8095C080C822C082D7CA292F092EE5
:10318000000C330B3F939F9382E492E09F938F93C5
:10319000FF92EF920E945C34F801EA5BFF4F80815E
:1031A000C82AC0820F900F900F900F900F900F9031
:1031B000BCCA85E691E01DCB2C9381E03DCD10E0AB
:1031C00081E0E9CA1F920F920FB60F9211248F93DC
:1031D0009F938091E1009091E100937F9093E100B3
:1031E00083FF0FC01092E90091E09093EB001092E2
:1031F000EC0092E39093ED0010925A0398E09093C4
:10320000F00082FF1CC093E09093E9009091F200DF
:10321000992319F09AE39093E80090914B03992336
:1032200029F090914B03915090934B039091590347
:10323000992329F09091590391509093590384FF59
:1032400018C08091E2008E7E81608093E2008091C0
:10325000E1008F7E8093E10080914C038E7E80613F
:1032600080934C039F918F910F900FBE0F901F90F2
:10327000189580FFF7CF8091E2008E7E8061809369
:10328000E2008091E1008E7E8093E10080914C030A
:103290008E7E8160E5CF1F920F920FB60F921124A0
:1032A000CF92DF92EF92FF920F931F932F933F9352
:1032B0004F935F936F937F938F939F93AF93BF933E
:1032C000EF93FF93CF93DF93CDB7DEB76C97DEBF5D
:1032D000CDBF1092E9008091E80083FF2FC089E004
:1032E000FE017596EE2EDF2E815029F09091F100AF
:1032F00090833196F9CF84E68093590382EF8093CF
:10330000E8008D8987FF39C09091E80090FFFCCFDD
:10331000982F907609F033C19E894F89588D2F8957
:10332000F88C911131C0803861F580914A03809307
:10333000F1001092F1008EEF8093E8006C960FB6CA
:10334000F894DEBF0FBECDBFDF91CF91FF91EF911B
:10335000BF91AF919F918F917F916F915F914F91AD
:103360003F912F911F910F91FF90EF90DF90CF90A1
:103370000F900FBE0F901F9018959EEF9093E8004E
:10338000C7CF1092F100D5CF913059F48111D3CF2E
:103390004130510581F680914A038D7F80934A0325
:1033A000CACF933049F48111C6CF4130510519F687
:1033B00080914A038260F2CF953041F48091E80019
:1033C00080FFFCCF20682093E300B5CF963009F052
:1033D000A8C00B8D1C8D22E01092E90010924803CA
:1033E00010924703F2122EC010924603109245032A
:1033F0000E9457071F8299E09983FA8291E09E8389
:1034000090EA98879AEF9987209147033091480373
:10341000275F3F4F3C832B838D831092E9001092EE
:10342000480310924703109346030093450349E075
:1034300050E0BE016F5F7F4F80E00E9431070E9425
:10344000570779CF10934603009345030E949406D3
:10345000DC0112960D911C910115110509F457C15B
:10346000D801ED91FC910480F581E02D6E2D7D2D2C
:10347000C8010995009709F045C1F801008511853B
:10348000EBCFF3E0FF120EC08F89882309F440C010
:10349000823061F440E867E184E69BE00E94811E8F
:1034A000811149CF81E28093EB0048CF813029F42C
:1034B00040E868E08BE59BE0F1CF833099F70E940C
:1034C0009406DC011296ED90FC908E010F5F1F4F69
:1034D0006801E114F10479F0D701ED91FC910680C7
:1034E000F781E02DB801C7010995080F111DF701FB
:1034F000E084F184EECFD8011C92F6010190002007
:10350000E9F73197BF016C197D0940E0C601C6CFCC
:1035100065E47BE0FB01449150E080E80E943107C4
:103520000ACF973009F4BECF983021F481E0809320
:10353000F10001CF993009F0FECE837009F0B2CFCF
:10354000E3E3F1E081E031E096E32191222371F0A1
:103550008093E9003093EB00DF0111972C912093C9
:10356000EC009093ED008F5F873079F78EE78093C2
:10357000EA001092EA008F8980935A03DCCE8B8D8B
:103580009C8D1092E900109248031092470390938B
:10359000460380934503898D81119AC08E899D8948
:1035A000913A49F4813209F07DCF47E050E064E080
:1035B00071E080E0B3CF913209F074CF833269F4C7
:1035C0008F89988DB0E0A0E0809300019093010175
:1035D000A0930201B0930301AECE8032A9F4809192
:1035E000E80082FFFCCF88E0E4E0F1E0815029F0C0
:1035F0009091F10090833196F9CF84E6809359033E
:103600008BEF8093E80097CE823209F094CE8F89B9
:1036100080930B01EEEFFFE7859194918B3F9C4DDA
:1036200051F1E0E0F8E08091040190910501A09152
:103630000601B0910701803B9440A105B105F1F46A
:1036400080910B0180FD1AC0EE3F8AE0F80789F5F2
:1036500087E797E791838083809160008093490397
:1036600088E19BE00FB6F894A895809360000FBEA8
:103670009093600060CEEEEFFAE0D5CF808191812B
:103680008737974709F057CEA895809160008861E9
:10369000809360008091490380936000EE3F2AE0B0
:1036A000F20789F08091FE0A9091FF0A918380834E
:1036B00042CE808191818737980751F29093FF0A1B
:1036C0008093FE0AC5CF1092FF0A1092FE0A33CEF5
:1036D0000E949406DC0112960D911C9101151105B2
:1036E00009F4E0CED801ED91FC910190F081E02D3C
:1036F0006E2D7D2DC801099581111DCEF801008523
:103700001185ECCF181619060CF415CECBCEF1E0CE
:10371000FF12B7CE69E47BE0FDCE1F920F920FB689
:103720000F9211242F933F938F939F93AF93BF9347
:1037300080911A0290911B02A0911C02B0911D026F
:103740003091190223E0230F2D3758F50196A11D62
:10375000B11D2093190280931A0290931B02A0932B
:103760001C02B0931D0280911E0290911F02A09135
:103770002002B09121020196A11DB11D80931E026D
:1037800090931F02A0932002B0932102BF91AF91AA
:103790009F918F913F912F910F900FBE0F901F908F
:1037A000189526E8230F0296A11DB11DD2CF1F92B6
:1037B0000F920FB60F9211242F933F934F935F9365
:1037C0006F937F938F939F93AF93BF93EF93FF93E9
:1037D0008091B900887F803609F44AC0F0F58832BC
:1037E00009F4A5C018F5803109F499C0B8F488230C
:1037F00009F4F2C0883009F492C0FF91EF91BF91B3
:10380000AF919F918F917F916F915F914F913F9178
:103810002F910F900FBE0F901F901895883109F4CB
:1038200086C0803251F78093800314C0803409F43D
:103830009BC040F48033B9F38833F9F6809380035A
:1038400085ECAEC0803509F483C0883509F494C096
:10385000883499F60E946709D0CF883909F48AC064
:1038600038F5883729F050F4883611F0803729F67A
:1038700083E0809382031092180255C0883809F4BF
:1038800079C0803919F0803809F0B7CF80911802DB
:10389000803208F06FC0E091180281E08E0F8093B3
:1038A00018028091BB00F0E0E850FE4F80833BC0DF
:1038B000803B39F0D0F4803A09F477C0883A09F0B7
:1038C0009CCF84E0809382031092F7011092F6015E
:1038D000F0E0E0E009958091F60181110FC081E0F0
:1038E0008093F6011092D60109C0803C09F4A8CF5C
:1038F000883C09F4A5CF883B09F07FCFE091F70120
:1039000081E08E0F8093F701F0E0EA52FE4F808154
:103910008093BB009091F7018091F60129C08091BE
:103920005D038093BB0085EC8093BC0066CF9091D3
:103930007F0380917E03981758F5E0917F0381E023
:103940008E0F80937F03F0E0E25AFC4F8081E9CF35
:10395000E0917F0381E08E0F80937F038091BB0015
:10396000F0E0E25AFC4F808390917F0380917E03C8
:103970009817C8F285E8D8CFE0917F0381E08E0FD9
:1039800080937F038091BB00F0E0E25AFC4F80837C
:103990008091810381115ECF81E080935C0384EA92
:1039A0008093BC001092820328CF8091180280324D
:1039B00030F4E0911802F0E0E850FE4F10820E94CF
:1039C00067096091180270E088EF91E0F0E0E0E0B4
:1039D00009951092180234CF109280033BCF1F92AA
:1039E0000F920FB60F9211242F938F939F93EF9303
:1039F000FF938091C8009091C9002091CE008C71F6
:103A000079F491FD0DC08091AA019091AB01FC0168
:103A1000E957FF4F208388579F4F21E0FC01208307
:103A2000FF91EF919F918F912F910F900FBE0F906B
:103A30001F9018951F920F920FB60F9211242F937B
:103A40003F934F935F938F939F93AF93BF93EF9366
:103A5000FF938091AA019091AB01FC01EA57FF4FBF
:103A600020812223C9F18C579F4FDC01ED91FC91FD
:103A7000208131818091C90030FF2CC0816080930A
:103A8000C9002093CE002091AA013091AB01F90129
:103A9000EA57FF4F808181508083329780819181E6
:103AA0000296A9014E575F4F8417950710F0C90180
:103AB000029691838083FF91EF91BF91AF919F9187
:103AC0008F915F914F913F912F910F900FBE0F906B
:103AD0001F9018958E7FD3CF8091C9008F7D806411
:103AE0008093C900E091AA01F091AB01E757FF4F25
:103AF0001082E1CF1F920F920FB60F9211248F9375
:103B0000EF93FF93E9ECF0E08081877B806980830D
:103B1000FF91EF918F910F900FBE0F901F9018950E
:103B20001F920F920FB60F9211242F938F939F9392
:103B3000EF93FF93809171008B7F80937100809150
:103B400091008F7B80939100809124022091A901A4
:103B500020589091A801893020F49695922B8F5F80
:103B6000FACF9093A801809142028F5F843108F0D0
:103B700080E020914102281739F0E82FF0E0E35D62
:103B8000FD4F908380934202109224028091910015
:103B90008F7B809391001092A901FF91EF919F91EB
:103BA0008F912F910F900FBE0F901F9018951F921D
:103BB0000F920FB60F9211242F933F934F935F9361
:103BC0006F937F938F939F93AF93BF93EF93FF93E5
:103BD00080919600909197004091A90120919100C9
:103BE0004423F1F12F7B209391001092A901309191
:103BF000240231113CC0411122C020912502309194
:103C00002602280F391F30939B0020939A0024E04E
:103C100028BB20917100246020937100209127021D
:103C200030912802820F931F36952795280F391F50
:103C30003093A7012093A60181E080932402FF9195
:103C4000EF91BF91AF919F918F917F916F915F9114
:103C50004F913F912F910F900FBE0F901F9018958D
:103C600020642093910020E82093A901C0CF4091C7
:103C7000A6015091A7016091270270912802DB01F3
:103C8000A095B095E091A9012091A801841B950B06
:103C9000A817B90768F126952E2B460F571F3F5FCF
:103CA000861B970B3930A0F32093A80180917100F7
:103CB0008B7F80937100809142028F5F843108F086
:103CC00080E090914102981749F0E82FF0E0909140
:103CD000A801E35DFD4F90838093420280919100A3
:103CE0008F7B809391001092A90110922402A7CF9C
:103CF0002093A8015093A7014093A601309324027A
:103D00009ECFEF92FF920F931F93CF93DF93F82EE6
:103D1000192FE62E042F81E0860F880F0E940307DB
:103D200083E00E940307CF2DD12FEC0EFD2EF11C56
:103D3000CE15DF05B9F007FF13C0FE0184910E9484
:103D40000307182F80E00E94030781232196811129
:103D5000EFCFDF91CF911F910F91FF90EF900895DA
:103D60008881EDCF81E0F5CFE9EFF3E01382128295
:103D700088EE93E0A0E0B0E084839583A683B783C8
:103D80002DE331E0318320832FEF3FEF3587248708
:103D9000E9E4F4E01382128284839583A683B783D7
:103DA0008FE491E0918380830895CF93DF93CDB723
:103DB000DEB7EE970FB6F894DEBF0FBECDBF789496
:103DC00084B5826084BD84B5816084BD85B5826020
:103DD00085BD85B5816085BD80916E0081608093D1
:103DE0006E0010928100809181008260809381003A
:103DF000809181008160809381008091800081604A
:103E000080938000809191008260809391008091E6
:103E100091008160809391008091900081608093F7
:103E200090008091C10084608093C1008091C100A6
:103E300082608093C1008091C10081608093C10045
:103E40008091C30081608093C3008091C000826034
:103E50008093C0008091C20081608093C2008091F5
:103E60007A00846080937A0080917A0082608093E7
:103E70007A0080917A00816080937A0080917A0044
:103E8000806880937A0010925A0310924A0310922D
:103E90004C038091D70081608093D70080EA8093A3
:103EA000D80089B5806189BD89B5826089BD09B4B2
:103EB00000FEFDCF61E070E080E090E00E94A50888
:103EC0008091D8008F7C80618093D8008091E00041
:103ED000807F8093E0008091E1008E7E8093E100FE
:103EE0008DE08093E20060E080E00E94D01161E00C
:103EF00080E10E942B0810E001E0812F86958695D5
:103F00008695682E712C212F27702AA3F301EC527D
:103F1000FD4F808190E002C0959587952A95E2F744
:103F200080FF67C11C3108F0DAC0103110F00C942A
:103F3000D3271F3010F00C949F27143008F41DC1B4
:103F40008091410390914203892B09F074C08FEB5B
:103F500090E00E94EB32FC018FEBDF011D928A950D
:103F6000E9F7168E178E11A210A212A213A214A2A4
:103F700015A216A210A617A211A612A613A614A681
:103F800015A617A616A610AA11AA12AA13AA14AA51
:103F900016AA15AA17AA10AE11AE12AE13AEDF0103
:103FA000A05CBF4F1C9211961C92119716961D9201
:103FB0001D921D921C9219971E961C9211961C928E
:103FC000119716961D921D921D921C9219971E967E
:103FD0001C9211961C92119716961D921D921D927D
:103FE0001C9219971E961C9211961C921197169668
:103FF0001D921D921D921C9219971E961C9211964D
:104000001C92119716961D921D921D921C92199743
:104010001E961C9211961C92509682E08C931196DB
:104020001C9211961C9211961C9252971C92F0931E
:104030004203E0934103E0904103F09042036701A3
:10404000BBE9CB0ED11CF60180819181892B09F04F
:10405000B8C081E090E00E94EB32D6018D939C9332
:104060001092710010929000B1E8B0939100E3E8D3
:10407000F6E0F0932802E09327027BE3A72E7CE38F
:10408000B72EB0922602A092250262E08DE00E9437
:104090002B0861E085E00E94FD0761E085E00E9459
:1040A0002B0810922402109242021092410280E2E8
:1040B00088BB809371006AE070E080E090E00E942D
:1040C000A508F701E156FF4F84E1810F8083319607
:1040D000A4EFCA2EDD24D394D182C08272C01232E2
:1040E00011F40C94112948F41F3108F4C7C71F318B
:1040F00011F40C94112980E065C0153211F40C9470
:104100001129C8F3A8EDEA2EE10E33E03E1598F32D
:1041100084E090E00E94EB325C01DC011C9213967B
:104120001C92F12CF701EE0FFF1FEA5AFD4F91830D
:10413000808382E090E00E94EB326C01FC011082EF
:104140001182D50112969C938E931197F701E75C2B
:10415000FC4F8081882379F2F601808362E00E941F
:104160002B08D6018C910E94D407F60181838AE046
:10417000810FD50113968C9324C0D090D402D3FA2A
:10418000DD24D0F88091430390914403892B81F47E
:1041900085E390E00E94EB32FC0185E3DF011D9294
:1041A0008A95E9F7118A128AF0934403E093430356
:1041B000E0904303F0904403F70184A9882309F4B5
:1041C0005BC681E0909155029F5F9093550221E07C
:1041D00030E00AA002C0220F331F0A94E2F7F30175
:1041E000E258FD4F882311F40C941C298081822B06
:1041F00080831F5F1C3209F080CE6DEF7AE08E0164
:104200000F5F1F4FC8010E9440348091DA028695EB
:1042100024ED32E03093A8032093A70322EF36E089
:104220003093B1032093B0039DE29093B4031093B5
:10423000AD030093AC03F80101900020E9F731973A
:10424000E01BF10BE093AE038093AF03882319F0DA
:10425000EF5FE093AE0384EB90E00E94EB329C01B1
:104260002C543F4FFC014FEF5FEFBA014193519344
:1042700061937193E217F307C9F79093B3038093A7
:10428000B2038AE890E00E94EB322AE8FC01119226
:104290002A95E9F728E231E0DC012D933C939093D5
:1042A000B8038093B7030E94C40C81E090E0909320
:1042B000AA038093A9038091DA0280FF0AC088E1F3
:1042C0009FE00FB6F894A895809360000FBE90937E
:1042D0006000A895209043033090440321143104DA
:1042E00059F10E945B09F101058516852785308902
:1042F0006017710782079307F8F08189813009F40C
:10430000A7C708F4A0C7823009F4B2C7D1015196FB
:104310008C9151978F5F51968C93882311F40C9454
:10432000542A0E945B09665F7F4F8F4F9F4FF101B8
:10433000658776878787908B0091410310914203B0
:104340000115110509F44AC0909142028091410281
:10435000981711F40C94632A8F5F843108F080E081
:10436000E82FF0E0E35DFD4F908180934102892FBB
:10437000582EBFEF8B1791F1F801E756FF4F7F01E1
:10438000980129573F4F690134E2831711F40C94C7
:10439000082C381714F40C94672A4AE0841721F08B
:1043A0005DE085130C941A2CD701EC9198012856E6
:1043B0003F4F3901EF3010F40C94772A412CF30170
:1043C00080818F5F8083D7011C9281E0BAE25B120B
:1043D00080E0F601808341100C94342C0E94800808
:1043E00000913D0310913E0320913F033091400323
:1043F000601771078207930708F428C50E94800898
:10440000605F784D8F4F9F4F60933D0370933E03E5
:1044100080933F039093400380918D02882341F065
:10442000815080938D02811103C081E00E9410129F
:1044300000914303109144030115110511F40C94EC
:104440009A2DD801D4968C91D497882359F05296FE
:104450009C9152979F3F31F4815011F40C943E2C63
:10446000D4968C93F801F081FAA700917C02109108
:104470007D020115110549F1D8011B968C911B97FE
:104480008823F1F015962D913C91243FB1E03B0734
:1044900010F00C949D2D2F5F3F4FF801368325833C
:1044A000838194810E94B50ABC0190E080E00E9463
:1044B000DB38D80117966D937D938D939C931A9753
:1044C000F8018081FAA5F82BFAA794E6E92E92E08C
:1044D000F92E22E3D22ED7010D911D917D010115F8
:1044E000110539F0F8018085815011F40C94362EB5
:1044F0008087ECE7F2E0EE15FF0569F70EE512E0C4
:104500001FA70EA71801D1010D911D911D010115C5
:10451000110509F491C0F801848D882309F48CC039
:104520008091940290E0218902C0959587952A9503
:10453000E2F780FF15C0E08924E0E29FF00111243A
:10454000EA54FD4F1082118212821382D8015796CD
:104550001C921E92569780918E02816080938E02EB
:10456000F801858D882309F460C08150858F811101
:104570005CC0828593850E94B50AD8015096EC9064
:10458000F12CBC0190E080E00E94DB38F80124852A
:104590003585468557850E94343A0E94AC3890E0B4
:1045A00080E00E94DB384B015C01F701E95EFC4FC3
:1045B00060816E5970E090E080E00E94DD3820E07C
:1045C00030E048EC52E40E9433382B013C01F70103
:1045D000EE0FFF1FEE53FD4F6081718190E080E090
:1045E0000E94DB389B01AC01C301B2010E94343A46
:1045F0009B01AC01C501B4010E94F33987FD15C0D0
:10460000F701EE0FFF1FEE0FFF1FEA54FD4F108260
:10461000118212821382D80157961C921E925697CD
:1046200080918E02816080938E02F801848D81508A
:1046300011F40C94542E848FE4E6F2E0E215F305B5
:1046400009F061CF209041033090420321143104DE
:1046500009F412C3F101E056FF4F80819181009768
:1046600031F0019711F40C94AF2E91838083F10106
:10467000E156FF4F8081815080838111F8C2D101C2
:104680008C9194E190838111D5C25F968C915F9754
:10469000882309F4CFC25E968C91882309F4CAC29C
:1046A0000E945B09F10104AD15AD26AD37AD601B6D
:1046B000710B820B930B613D77408105910508F0EA
:1046C000B9C28101025E1F4F1BA30AA3F101E65983
:1046D000FF4F11828681D10111968C93C8010E94EF
:1046E000890AF10162837383848395838AA19BA1E4
:1046F0000E945D0AD10116966D937D938D939C93D4
:104700001997F101EE55FF4F808181114CC08091C6
:10471000430291E0980F90934302893108F48AC2D2
:1047200081E080838AA19BA10E94890AF101ED5456
:10473000FF4F60837183828393837097608371835B
:10474000828393838AA19BA10E945D0AF101E954AF
:10475000FF4F60837183828393837097608371833B
:1047600082839383EB54F10911826681778180857E
:1047700091850E94DD3820E030E048EC52E40E9450
:1047800033380E94A538F101E554FF4F60837183EF
:104790008283938303571F4F0E94DD38F8016083A3
:1047A000718382839383F101E35AFF4F80818823D1
:1047B000F1F03197118266817781808591850E9421
:1047C000DD3820E030E048EC52E40E943338F1015B
:1047D000E555FF4F20813181428153810E944A3744
:1047E0000E94A538D1011B967C936E931A97F10114
:1047F000EF5BFF4F80818823B1F131971182668191
:104800007781808591850E94DD3826E53EE04DEE7A
:104810005FE30E94343A20E030E048EC52E40E942A
:1048200033380E94AC38F10175876487CB01B0E062
:10483000A0E04091AE025091AF026091B002709141
:10484000B102481759076A077B0768F48093AE02E4
:104850009093AF02A093B002B093B10280918E0208
:10486000816080938E02F101E15BFF4F808188239C
:10487000A9F03197118266817781808591850E94A8
:10488000DD3820E030E048EC52E40E9433380E94EA
:10489000AC38D10151967C936E9350978AA19BA11D
:1048A0000E945D0A5B016C018AA19BA10E94890A9A
:1048B0007B018C014101B7EA8B0E911CF401208130
:1048C000318142815381C1018D559F4F99AB88AB96
:1048D000DC016D917D918D919C910E94970E0E94BB
:1048E000AC38F101758B648B8AA19BA10E945D0A93
:1048F0002B013C018AA19BA10E94890A6B017C01CA
:10490000D4012D913D914D915C91C301B2010E9462
:104910004A3725E33AEF4EE85CE30E94343A4B0114
:104920005C0125E33AEF4EE85CE3E8A9F9A9608170
:104930007181828193810E94343A2B013C0125E3ED
:104940003AEF4EE85CE3C701B6010E94343A6B01CE
:104950007C01C501B4010E94F13A6CAB7DAB8EAB1A
:104960009FABC701B6010E942E3868AB79AB8AAB0A
:104970009BABC301B2010E94F13A68AF79AF8AAF35
:104980009BAFC501B4010E942E384B015C0128ADDC
:1049900039AD4AAD5BAD68A979A98AA99BA90E94E6
:1049A000343AA50194010E94343A4B015C01C301E1
:1049B000B2010E942E382B013C01C701B6010E94B2
:1049C000F13A9B01AC01C301B2010E94343AA50146
:1049D00094010E944A376B017C0128A939A94AA990
:1049E0005BA96CA97DA98EA99FA90E94343AA70151
:1049F00096010E94CA376B017C0120E030E0A901DA
:104A00000E94293887FF0AC02BED3FE049EC50E4B3
:104A1000C701B6010E944B376B017C0121EE3EE2DB
:104A200045E652E4C701B6010E94343A0E94AC3810
:104A3000D10153967C936E935297F101E554FF4F49
:104A400060817181828193810E94DD384B015C011C
:104A5000F101E45AFF4F118266817781808591854B
:104A60000E94DD3820E030E048EC52E40E94333808
:104A70006B017C01AC019B01C501B4010E94F339BB
:104A800087FF02C00C94CC2EA7019601C501B4018A
:104A90000E944A372B013C018AA19BA10E945D0A1A
:104AA0005B016C018AA19BA10E94890A7B018C0198
:104AB000F101E954FF4FF9ABE8AB2081318142812C
:104AC00053814101F3EB8F0E911CD4016D917D91C7
:104AD0008D919C910E94970E6B017C01A301920124
:104AE000C301B2010E94343A2B013C01A701960197
:104AF000C701B6010E94343A9B01AC01C301B20167
:104B00000E944B370E94FF3A6B017C0120E030E0AD
:104B100040E251E40E94F339810101551F4F1816FC
:104B20000CF07EC0F101E05CFF4F1182668177815D
:104B3000808591850E94DD3826E53EE04DEE5FE3FD
:104B40000E94343A20E030E048EC52E40E943338CE
:104B500020E030E040E251E40E94F33918160CF0F6
:104B60005FC0F80160817181828193810E94DB388E
:104B7000A70196010E944B370E94AC38D8016D9373
:104B80007D938D939C9313976091AA027091AB02D1
:104B90008091AC029091AD020E94DB38A701960192
:104BA0000E944B370E94AC386093AA027093AB020C
:104BB0008093AC029093AD0280918E0281608093CD
:104BC0008E028AA19BA10E94890AF40160837183ED
:104BD000828393838AA19BA10E945D0AA8A9B9A997
:104BE0006D937D938D939C931397F101E45AFF4F3E
:104BF00011827101BBEBEB0EF11C66817781808520
:104C000091850E94DD3820E030E048EC52E40E94BB
:104C100033380E94A538F7016083718382839383C0
:104C2000F80180819181A281B381F101868B978BFC
:104C3000A08FB18F6091AA027091AB028091AC02FB
:104C40009091AD022AE030E040E050E00E94543CF8
:104C5000D1015A962D933D934D935C935D9780912E
:104C6000AE029091AF021F969C938E931E97F10116
:104C70008081FAA5F82BFAA766E5A62E62E0B62E8B
:104C80007EE5C72E72E0D72EEAE09E2ED5010D916B
:104C90001D915D010115110539F0F80183818150E5
:104CA00011F40C94D22E8383CA14DB0479F780911B
:104CB000A9039091AA03009741F0019711F40C9475
:104CC000E72E9093AA038093A90380E00E9410121C
:104CD0008091550281110C9407318BEF9FEF9093D7
:104CE000540280935302809152028F5F8A3010F0F9
:104CF0000C941931809352028091930290E0880FB6
:104D0000892F881F990B892B79F087E00E94D4079F
:104D1000892B11F40C943131809194028F77809318
:104D2000940284E18093950280918E0280FF09C0F5
:104D30008E7F80938E0284EF91E090935002809357
:104D40004F0280914F0290915002009759F00197C5
:104D50009093500280934F02892B21F461E081E00F
:104D60000E94D01180914702282F082E000C330B8F
:104D7000909148029217130611F40C9444318093D9
:104D800048021092490210924A0210924B0210926D
:104D90004C028F3F49F11092490210924A02109240
:104DA0004B0210924C0210924E0210924D028091D2
:104DB0008E02826080938E028091490290914A0215
:104DC000A0914B02B0914C020097A105B10561F092
:104DD00091958195910990934E0280934D02809117
:104DE0008E02826080938E0280918B0290918C0261
:104DF00001971816190614F00C94583190938C02F0
:104E000080938B0210E000E08091830290E0002EFE
:104E100002C0959587950A94E2F780FF12C0F801C9
:104E2000EE0FFF1FEA5AFD4F0190F081E02D408107
:104E3000042E000C550B660B770B88E2800F0E9446
:104E4000ED050F5F1F4F04301105F1F680918E02C2
:104E500081FF0AC08D7F80938E0280918D02811127
:104E600003C08AE080938D0280E090E0892B09F4F2
:104E700030CA0E9400002DCAD7A2109223021092BD
:104E80002202109284031092A603109282030093D0
:104E9000810310925C0361E082E00E94FD0761E003
:104EA00083E00E94FD078091B9008E7F8093B90056
:104EB0008091B9008D7F8093B90088E48093B80019
:104EC00085E48093BC000093830387E78093A50368
:104ED000109284031092A6030E94000681110BC950
:104EE0006EE1C7010E94F50B64E670E080E090E09F
:104EF0000E94A5086701B3E1CB0ED11CF2EABF2ED8
:104F000042E050E06B2DC7010E94100CF601619346
:104F100071936F01B394B394FEEABF12F1CFA12C49
:104F2000B12C6501A394D7011D96AD92BD92CD928F
:104F3000DC92509784E1810FD4968C9342C98CE027
:104F400090E00E94EB326C01FC017CE0A72E1192F4
:104F5000AA94E9F790937D0280937C02DC011B9672
:104F60008C911B9781112DC9E3E21B96EC9383E092
:104F700090E00E94EB327C01DC011C9212961C92A4
:104F80001E921197F60194838383809126038823D0
:104F900009F4B1C88C930E945C08D70112969C93C7
:104FA0008E9311970EC989E090E00E94EB325C016C
:104FB000FC0159E0C52E1192CA94E9F780EF810FE8
:104FC000C82ED12C7601EE0CFF1CF701EC59FD4FD9
:104FD000B182A08283E090E00E94EB324C01DC01C0
:104FE0001C9212961C921E921197F5019383828354
:104FF000F601E35DFC4F8081882309F47CC88C9323
:105000000E945C08D40112969C938E931197F7012D
:10501000E257FD4F7F01E559FF4FC080D180F3E596
:10502000EF0EF11CD7016D917C916C0D7D1D90E010
:1050300080E00E94DB381B012C01BFEFCB1ADB0A9A
:10504000B60190E080E00E94DB389B01AC01C20118
:10505000B1010E94333820918F023091900240912B
:105060009102509192020E94343AF5016483758353
:105070008683978382E3810F8087A3C88EE190E0C7
:105080000E94EB327C01DC01EEE11D92EA95E9F72A
:1050900084EE810F282F30E0F901EE0FFF1FE25A56
:1050A000FD4FF182E082D70150968C93F901E257CF
:1050B000FD4F6F01ED57FF4F8081882309F41BC816
:1050C00083E090E00E94EB325C01DC011C921296BE
:1050D0001C921E921197F70191878087F601E7567F
:1050E000FF4F8081882341F08C930E945C08D5019A
:1050F00012969C938E93119783E090E00E94EB327E
:105100006C01FC01108212821182D7011B969C93C4
:105110008E931A975096EC91F0E0E65DFC4F8081FB
:10512000882349F0F60180830E945C08D60112961C
:105130009C938E931197F701C088D12CF601EE0F46
:10514000FF1FE05EFC4FA080B180F601EE0FFF1F55
:10515000E65EFC4F608171816A0D7B1D90E080E00E
:105160000E94DB381B012C01FFEFAF1ABF0AB5010B
:1051700090E080E00E94DB389B01AC01C201B101EC
:105180000E94333820918F02309190024091910219
:10519000509192020E94343AD7011C966D937D93F0
:1051A0008D939C931F97F601E95EFC4F80818130BF
:1051B000B1F562E087E00E942B088091930280683D
:1051C0008093930287E0F701818B808990E0FC0156
:1051D000E95EFC4F2081223020F0E8ECD7015D969B
:1051E000EC93880F991F880F991FFC01EA54FD4F1B
:1051F00020E030E040E251E460817181828193815E
:105200000E944B370E94AC38D70157967C936E931F
:10521000569784E1810F5C968C930C94E12080E09A
:10522000D2CF81E020915E0230915F02232B11F0FA
:105230000C94E2200C947B2000938A028681822BBE
:1052400086830C94F92068E4C1010E94F50B5EC8C6
:1052500043E050E060E0C1010E94100C609329021D
:1052600070932A0280932B0290932C0268E5ECCF76
:1052700043E050E060E0C1010E94100C2B013C01B2
:10528000D1015B968D919C91B0E0A0E0BA2FA92F3F
:10529000982F8827481A590A6A0A7B0AF101658DF6
:1052A000768D90E080E0A30192010E94063D07E127
:1052B0000E94593D49019A0184010053184F2F4F14
:1052C0003F4F0AA71BA72CA73DA7D10157966D9169
:1052D0007C9190E080E0A30192010E94063D08E0ED
:1052E0000E94593D2AA33EA74A01B62FA72F88AB9B
:1052F0009CABF101A388B488950140E050E060E0E8
:1053000070E080E090E00FE00E94403D59016A01AA
:105310007B018C012AA13EA5A4016B2F7A2F88A9BD
:105320009CA90E94763DA0902902B0902A02C090CC
:105330002B02D0902C0276016701E12CF12C870121
:10534000AAA2BBA2CCA2DDA2EEA2FFA208A719A727
:10535000E12CF12C00E010E00E94AE3C05E10E943F
:10536000593D2AA33EA74A0168AB7CAB88AF9CAFEE
:10537000D10159966D917C9190E080E0A30192015A
:105380000E94063D07E00E94593D29013A01B62FCF
:10539000A72F8DAF9EAFF101A588B688950140E09B
:1053A00050E060E070E080E090E000E10E94403D6D
:1053B00059016A017B018C019201A3016B2F7A2FA5
:1053C0008DAD9EAD0E94763D59016A017B018C0135
:1053D0002AA13EA5A40168A97CA988AD9CAD0E9424
:1053E0007F3D0FE00E94593D79018A01678D70A1D0
:1053F00081A192A10E94DD3820E030E040E45FE32B
:105400000E94343A4B015C01B701C8010E94DD38AB
:1054100020E030E040E85EE30E94343A9B01AC01BA
:10542000C501B4010E944B370E94A538D1015F9697
:105430006D937D938D939C93929752968C915297F6
:10544000823370F58F5F52968C9352975F96EC92F1
:105450005F979096FC92909791960C939197929665
:105460001C9392979396EC9293979496FC929497B0
:1054700095960C93959796961C938FEFD101519624
:105480008C936AA57BA58CA59DA52AE030E040E021
:1054900050E00E94763CF101328321830C948621F6
:1054A0008FEFF101828BE9CF0E945B09605B7F4F38
:1054B0008F4F9F4FD1011D966D937D938D939C933C
:1054C00050970C949C218FEF9FEF0C94B8217AE2B7
:1054D000871711F40C94D421ACE28A13ABC1F80104
:1054E000EA57FF4F9081892780830C94D421E00FE5
:1054F000F12FF11DE857FF4F1082D6014C90442048
:1055000009F4BFC0F801E857FF4F2081822F022E17
:10551000000C990B3FEB320F363008F053C0C797A1
:105520008295807FF801E757FF4F9081292F092E40
:10553000000C330B4FEB490F463008F04BC027539C
:105540003109820FF801EA57FF4F908189130C94BB
:10555000DE217196B080BB2009F445C0B1E0BB12DA
:105560000C94DF2133969080992011F40C94DF2164
:1055700087E0EC56F109D801909601900D928A953A
:10558000E1F787E0F801F596D801979601900D9222
:105590008A95E1F70E945B09F80164AF75AF86AFA9
:1055A00097AFB78EB68E5801FEE1AF0EB11CC501A4
:1055B00082960E94460AC501C0960E94460A492C5E
:1055C0000C94DF212156263018F487559109A8CF75
:1055D000C097A6CF9156963018F427553109B1CF10
:1055E00020533109AECFF801E656FF4F8081882362
:1055F00031F187E0EC56F109D801909601900D92B7
:105600008A95E1F787E0F801F596D8019796019021
:105610000D928A95E1F70E945B09D801DC966D93A3
:105620007D938D939C93DF9781E05F968C935F973A
:105630005E968C93C801845A9F4F0E94460A580177
:10564000BAE6AB0EB11CF50182859385A485B585BC
:1056500086839783A087B1870E945B09D501129644
:105660006D937D938D939C93159781E011968C9308
:1056700011978C93C80188589F4F0E94460A0C943A
:10568000DF21F9013081A80149565F4F5A013111DC
:105690002BC0480158E8850E911C6EE871E0C401EA
:1056A0000E94A73D892B39F064E971E0C4010E9492
:1056B000A73D892B29F481E0D5018C930C94DF213F
:1056C0006AE971E0C4010E94A73D892B39F060EAC4
:1056D00071E0C4010E94A73D892B21F4F5011082DD
:1056E0000C94DF2182E0E8CFDA01EC91E23011F492
:1056F0000C94DE21C80188579F4FDC012C91222396
:1057000011F40C94DE21B0E2EB9FF0011124E32BA5
:105710003297E732F10510F00C94DF21EE56F44D8C
:105720000C94953CC12BC82BD02BD42BEA2BF32BFC
:10573000FE2B032CDF21DF21DF21DF21DF21DF2111
:10574000DF21DF21DF21DF21DF21DF21DF21DF2159
:10575000DF21DF21DF21DF21DF21DF21DF21DF2149
:10576000DF21DF21B92BC12BC82BD02BD42BDD2B74
:10577000E52BF801E656FF4F81E0213489F180E006
:105780002FC0B801625D7F4F0E94D80F0C94DF21BB
:1057900081E0233509F080E0F80184AB0C94DF212F
:1057A000B8016B5C7F4FF0CF81E0273509F080E0D6
:1057B000D801DB968C930C94DF21BC01C801805C7E
:1057C0009F4F0E947B0F0C94DF21BC01C801825BBC
:1057D0009F4FF7CFF801E656FF4F81E021337CF26F
:1057E00080830C94DF210E941034F801E659FF4FAA
:1057F00062877387848795870C94DF21BC01C80179
:1058000088589F4FDECFBC01C801845A9F4FD9CF23
:105810001082F801E856FF4F10827297108271963D
:1058200082E08083F6011082F801E656FF4F108275
:105830000C94EE21D701EC91EE3048F481E08E0F0C
:105840008C93E00FF12FF11DE857FF4F5082F601C6
:10585000808181110C94EE21F801EA57FF4F80817D
:10586000582650820C94EE21F801E356FF4F8081B8
:1058700091810196918380830C94EE2184E1F8015B
:1058800084AB678D70A181A192A10E94DD386B016C
:105890007C01D80193966D917D918D919C91969705
:1058A0000E94DD389B01AC01C701B6010E9433386C
:1058B0002BEA3CED42E45EE30E94A13A9B01AC017D
:1058C00060E070E080E89FE30E944A3720E03AE21F
:1058D0004DE257E40E94343A0E94A538F8017483DF
:1058E000638323853485A901465F5F4F46175707B9
:1058F0000CF000C1621B730BCB01770FAA0BBB0B23
:105900004091B2025091B3026091B4027091B5021D
:10591000840F951FA61FB71F8093B2029093B30206
:10592000A093B402B093B50280918E0281608093FF
:105930008E0283819481948783876091B2027091F3
:10594000B3028091B4029091B50228EE33E040E0BA
:1059500050E00E94543CF8012583368347835087EA
:1059600087A1882311F40C943222678D70A181A144
:1059700092A10E94DD386B017C01D80193966D9154
:105980007D918D919C9196970E94DD389B01AC0191
:10599000C701B6010E9433382BEA3CED42E45EE3D6
:1059A0000E94A13A9B01AC0160E070E080E89FE3B7
:1059B0000E944A3720E03AE24DE257E40E94343A2E
:1059C00020E030E048EC52E40E94343A0E94A538CE
:1059D0004B015C01F801C4A4D5A4E6A4F7A4C1144A
:1059E000D104E104F10459F10E945B09D801D09679
:1059F0004D905D906D907C90D397641975098609E0
:105A000097090E94DB389B01AC0160E070E08AE7F7
:105A100094E40E9433382B013C01C501B4016C1998
:105A20007D098E099F090E94DD389B01AC01C301ED
:105A3000B2010E94343A0E94A5386B017C01F80142
:105A400084A695A6A6A6B7A60E945B09D801D09603
:105A50006D937D938D939C93D39798966D917D9143
:105A60008D919C919B976C197D098E099F090E94CD
:105A7000DD384B015C016091DF0270E090E080E076
:105A80000E94DD3820E030E048EC52E40E943338D8
:105A90009B01AC01C501B4010E94343A4B015C0189
:105AA000C701B6010E94DD389B01AC01C501B401FC
:105AB0000E944B370E94A538F80160A771A782A702
:105AC00093A7C090E0028C2C912CB12CA12C8616AF
:105AD0009706A806B906C4F46B017C01C818D9085A
:105AE000EA08FB084601D8011A969C928E921997F3
:105AF0000C943222AB01465F5F4F421753070CF004
:105B00001CCF7487638719CFD12CD194C194D1084D
:105B10000D2C000CEE08FF086C157D058E059F0509
:105B20002CF4860E971EA81EB91EDDCF812C912C59
:105B30005401D9CF1AA60C943522815021F0F801D6
:105B400083870C94602284E1D8011B968C931B9769
:105B500013968D919C910E94B50ABC0190E080E063
:105B60000E94DB3820E030EC4AE754E40E94F3392D
:105B700087FD07C0F8011282118281E080830C94B6
:105B80006022D8011C9248E0C42ED12CF12CE12CCB
:105B9000F801838194810E94B50AE80EF91EF1E0B4
:105BA000CF1AD108A9F733E0F594E7943A95E1F7D5
:105BB000D80117968D909D90AD90BC901A97B70123
:105BC0000F2C000C880B990B0E94DD38A501940165
:105BD0000E94293887FF05C0C501B4010E94A5387D
:105BE0007B01B701FF0C880B990B0E94DD38A501E2
:105BF00094010E944A3720E030E040E85AE30E94D6
:105C0000343A20E030E44CE955E40E94343A20E88C
:105C100036EE45EC57E40E944B3720E836EE45EC73
:105C200057E40E944A379B01AC010E944B372CE19C
:105C30003EE14AE95FE30E9433380E94FF3A26E6DC
:105C400036E646E650E40E94343A0E94AC386431AD
:105C5000710528F0F801728361830C946022D801E9
:105C600012961C921E9211970C946022D08682810B
:105C700093810E94B50ABC0190E080E00E94DB386D
:105C8000F80124813581468157810E94343A20E011
:105C900030E040E251E40E9433380E94AC38D80131
:105CA0006D937C930C947922E4E1D8015C96EC939B
:105CB00060E0C8010E94F30A4B015C01D8011A960A
:105CC0008D919C910E94B50ABC0190E080E00E94F9
:105CD000DB38F80124853585468557850E94343A9E
:105CE0000E94AC386B01C501B4010E94DB3820E092
:105CF00030E040E251E40E9433380E94AC38D801D1
:105D00006D937C93712C612CC301B6010E94DB382A
:105D100020E030E040E251E40E9433380E94AC3889
:105D2000F80173836283A3019601C501B4010E9447
:105D3000303C20E432E44FE050E00E94543CD80173
:105D400015963C932E9314975096EC91F0E0EE0F3D
:105D5000FF1FEE53FD4FD182C0820C941C2384EFB1
:105D600091E091838083F101E356FF4F808191811F
:105D700020914402309145028217930750F421E0AC
:105D8000D1012C93449690934502809344020C9445
:105D90003723F1011082F6CFA5019401C701B601A6
:105DA0000C9448259382E180F280F701808188235A
:105DB00029F00E94D407D70111968C9381E0F70156
:105DC0009181911180E0D8018C930C9454268FE03E
:105DD00090E09093AA038093A9038091B0039091DF
:105DE000B103892B09F4C8C18091AB0391E0980FEE
:105DF0009093AB03811154C01092BB031092C10366
:105E0000F090AE038F2D880F880F880F8093C20308
:105E10000F2D10E06091AC037091AD03A80183ECED
:105E200093E00E94973D8091AF03882329F0F80109
:105E3000E955FC4F8063838F1AE01F0D8EE7809336
:105E4000B9038FE28093BA038091BB039EEF910F59
:105E5000892B8093BB0389E08093BC0384EA809301
:105E6000BD038091AF038F5E8093BE0383E2809376
:105E7000BF031092C003E12FF0E0ABEBB3E092E080
:105E800080E037E0911708F03FC12D91822728E08C
:105E900087FF38C1880F83272150D1F79F5FF2CF4A
:105EA0002091B403982F9695291708F445C080FDDA
:105EB00043C010E000E08091B4038017110609F0A0
:105EC0000CF41EC16091B60370E0CE0101960E94F1
:105ED000530D8091B6038F5F8093B6039091B40306
:105EE000891710F01092B6038885882311F110925B
:105EF000BB038B818093C1038D8DB8E08B9F900194
:105F000011248E8D822B8093C20380E01AE0180F3B
:105F1000E9E0F0E0EC0FFD1FE80FF11D90819923FF
:105F200009F48CCF8F5FE12FF0E0E754FC4F9083B2
:105F3000EDCF0F5F1F4FBFCF80E48093BB03F12CE9
:105F4000E12C18E06091B50370E0CE0101960E944B
:105F5000530D8091B5038F5F8093B5039091B40387
:105F6000891710F01092B5038885882309F4C5C0FD
:105F70008C819D81AE81BF818F3FEFEF9E07AE0781
:105F8000BE0709F4BAC0E12FF0E04B813F8D21E05C
:105F9000210FE955FC4F632F6F704031A8F0628BE1
:105FA000E22FF0E0E955FC4F428B22E0210F69A17E
:105FB00070E0343009F45FC070F4332339F13130CC
:105FC00009F446C010E02EC000E1409FA00111245A
:105FD000462B428BECCF383009F464C0393009F4D9
:105FE00079C0353079F7422F50E0FA01E754FC4F81
:105FF0008083FA01E654FC4F908345545C4F3B2F5D
:106000003078832F8A2BDA018C934AC0E22FF0E09C
:10601000E754FC4F3B2F30788F71832B98A1892B4D
:10602000808311E0120FFFEFEF1AFF0A812F90E03B
:106030002091B4032E151F0409F00CF4FFCE2AE1C1
:1060400030E0261B370B821793070CF47BCFF6CE7C
:10605000422F50E0FA01E754FC4F808346545C4FD6
:10606000392F3F718B2F8078832B98A1892BDA01F0
:106070008C9312E0D7CF422F50E0FA01E754FC4F47
:106080008083FA01E654FC4F908345545C4F3A2FCD
:106090003F718B2F8078832B98A1892BFA01808305
:1060A00013E0C0CF422F50E0FA01E754FC4F808349
:1060B000FA01E654FC4F9083FA01E554FC4FA083AB
:1060C00044545C4F8B2F8F7998A1892BFA018083E0
:1060D00014E0A8CF422F50E0FA01E754FC4F808330
:1060E000FA01E654FC4F9083FA01E554FC4FA0837B
:1060F00044545C4FFA01B083EBCF70E060E093CF83
:1061000010E09CCE880FC8CEE955FC4F828B809161
:10611000B7039091B803DC01ED91FC910280F3810B
:10612000E02D40E06EE7099501E08091B703909182
:10613000B803101788F0A02FB0E0A955BC4FFC01A0
:1061400020813181F9012281338141E052966C91A5
:10615000F90109950F5FE9CF80914602853860F417
:106160008F5F809346028091AB0386959091B40334
:10617000981710F41092AB038091B7039091B80375
:10618000DC01ED91FC910280F381E02D40E06EEFA7
:1061900009958091D903882339F109ED13E059EF6E
:1061A000E52E53E0F52E8091B7039091B803F801E6
:1061B00061918F01DC01ED91FC910280F381E02D72
:1061C00041E00995E016F10671F78091B7039091CF
:1061D000B803DC01ED91FC910280F381E02D40E0F9
:1061E0006FEF09950C94652600E210E08091B703EB
:1061F0009091B803DC01ED91FC910280F381E02DD8
:1062000041E060E009950150110981F7DECF8091EE
:106210008A02882321F085E595E50C946F26BAA5BE
:106220008FEF90E0B1110C946F2681E090E00C9418
:106230006F26109252021091510260915302709198
:106240005402012E02C0769567950A94E2F76170B8
:1062500080E10E94FD071F5F1F70109351020C9494
:106260007C2680919502882311F40C949426815009
:106270008093950281110C949426809194028068F9
:10628000809394020C9494268F3F11F40C94F4267E
:106290008091490290914A02A0914B02B0914C0228
:1062A000892B8A2B8B2B11F00C94DC260C94CB269B
:1062B0008AE090E090938C0280938B02E0907E02C3
:1062C000E0FE0DC0E0914303F0914403438154810B
:1062D000052E000C660B770B80E00E94ED05E1FEB9
:1062E0000BC0E0914303F0914403458156816781DF
:1062F000708581E00E94ED05E2FE0DC0E091430350
:10630000F091440341815281052E000C660B770BFE
:1063100082E00E94ED05E3FE0DC0E0914303F091A1
:10632000440341855285052E000C660B770B83E0F4
:106330000E94ED05F0907F02F7FE0BC0E0917C0219
:10634000F0917D024181528170E060E08FE00E9417
:10635000ED0500E110E0D12CC12CF80133E0F595FA
:10636000E7953A95E1F7E258FD4F808190E098017A
:106370002770332702C0959587952A95E2F780FF0D
:1063800018C0F801EE0FFF1FEC5BFD4FA080B1803D
:10639000F501408151814C195D0970E060E0802F6A
:1063A0000E94ED058091DB0280FF03C0D501CD90F6
:1063B000DC900F5F1F4F0C31110579F605E210E0FC
:1063C0008091810290E098012152310902C0959597
:1063D00087952A95E2F780FF0CC0AEA5BFA5ED9189
:1063E000FC914081518170E060E087EF800F0E9456
:1063F000ED05980126503109F90193E0F595E795EF
:106400009A95E1F7E258FD4F808190E0277033279D
:1064100002C0959587952A95E2F780FF0CC0AEA53E
:10642000BFA5ED91FC914281538170E060E08AEF5D
:10643000800F0E94ED05C0908202D12CC801839785
:10644000F60102C0F595E7958A95E2F7E0FF0CC0EA
:10645000AEA5BFA5ED91FC914481558170E060E04F
:106460008DEF800F0E94ED05C8018770992702C04B
:10647000D594C7948A95E2F7C0FE0BC0AEA5BFA520
:10648000ED91FC914681578170E060E0802F0E9481
:10649000ED050F5F1F4FEEA5FFA53296FFA7EEA7F4
:1064A0000832110509F08CCFE4FE0BC0E0914103E6
:1064B000F0914203418150E070E060E084E00E948E
:1064C000ED05E5FE0CC0E0914103F091420322810D
:1064D00033814481558160E085E00E94F20CE6FE44
:1064E0000CC0E0914103F091420326813781408541
:1064F000518561E086E00E94F20CE7FE0DC0E0915C
:106500004103F091420342855385052E000C660B32
:10651000770B87E00E94ED05F0FE0BC0E091410390
:10652000F09142034485558570E060E088E00E9468
:10653000ED05F1FE0BC0E0914103F0914203468569
:10654000578570E060E089E00E94ED05F2FE0BC027
:10655000E0914103F09142034089518970E060E08D
:106560008AE00E94ED05F3FE0BC0E0914103F0913B
:1065700042034289538970E060E08BE00E94ED05A0
:10658000F4FE0BC0E0914103F09142034489558928
:1065900070E060E08CE00E94ED05F5FE0BC0E0913C
:1065A0004103F091420346895789608D718D8DE0DA
:1065B0000E94ED05F6FC02C00C940227E091410315
:1065C000F0914203428D538D648D758D8EE00E9453
:1065D000ED050C9402270F931F93CF93DF93823026
:1065E000910510F482E090E0E0915704F091580496
:1065F00030E020E0B0E0A0E0309799F421153105BB
:1066000009F44AC0281B390B24303105D8F58A819A
:106610009B816115710589F1FB0193838283FE01E2
:1066200011C0408151810281138148175907E0F060
:106630004817590799F4109761F012960C93129726
:1066400013961C933296CF01DF91CF911F910F913A
:1066500008950093570410935804F4CF2115310581
:1066600051F04217530738F0A901DB019A01BD012F
:10667000DF01F801C1CFEF01F9CF90935804809367
:106680005704CDCFFE01E20FF31F81939193225067
:10669000310939832883D7CF20915504309156048E
:1066A000232B41F420910E0130910F0130935604B9
:1066B0002093550420910C0130910D0121153105D5
:1066C00041F42DB73EB74091100150911101241BA8
:1066D000350BE0915504F0915604E217F307A0F44E
:1066E0002E1B3F0B2817390778F0AC014E5F5F4F28
:1066F0002417350748F04E0F5F1F50935604409300
:106700005504819391939FCFF0E0E0E09CCFCF932D
:10671000DF930097E9F0FC01329713821282A09177
:106720005704B0915804ED0130E020E01097A1F437
:1067300020813181820F931F20915504309156049E
:106740002817390709F061C0F0935604E093550407
:10675000DF91CF910895EA01CE17DF07E8F54A816E
:106760005B819E0141155105B1F7E901FB83EA8385
:1067700049915991C40FD51FEC17FD0761F4808131
:1067800091810296840F951FE90199838883828104
:1067900093819B838A83F0E0E0E012968D919C9137
:1067A00013970097B9F52D913C911197CD01029661
:1067B000820F931F209155043091560428173907F2
:1067C00039F6309751F51092580410925704B0934F
:1067D0005604A0935504BCCFD383C283408151811A
:1067E000840F951FC817D90761F44E5F5F4F8881EA
:1067F0009981480F591F518340838A819B819383DC
:1068000082832115310509F0B0CFF0935804E0934D
:1068100057049ECFFD01DC01C0CF13821282D7CF77
:106820001F93FC0199278827BC01E894119110322D
:10683000E9F3193010F01E30C8F31B3251F01D324D
:1068400049F4689406C00E944734610F711D811D90
:10685000911D119110531A30B0F33EF4909580952C
:10686000709561957F4F8F4F9F4F1F910895FB014A
:10687000DC0102C005900D9241505040D8F70895B8
:10688000FB01DC0105900D920020E1F70895592FDE
:10689000482F372F262F660F771F881F991F660FE7
:1068A000771F881F991F620F731F841F951F660F24
:1068B000771F881F991F0895AEE0B0E0E2E6F4E389
:1068C0000C9421370D891E898EE08C831A830983ED
:1068D0008FEF9FE79E838D83AE01475E5F4F6F8989
:1068E000788DCE0101960E947F342F813885020F6A
:1068F000131FF80110822E96E4E00C943D37ABE0B4
:10690000B0E0E5E8F4E30C9413377C013B018A0125
:10691000FC0117821682838181FFC8C1CE010196D6
:106920005C01F7019381F30193FD859193FF8191C0
:106930003F01882309F453C1853239F493FD8591D1
:1069400093FF81913F01853229F4B70190E00E94C5
:106950006F36E7CF912C212C312CFFE1F31538F065
:106960008B3211F190F4803209F1833229F137FC36
:106970003CC020ED280F2A3050F536FE20C08AE0BA
:10698000989E200D1124922E06C08D3291F08033F6
:1069900071F7689430F8F30193FD859193FF81912D
:1069A0003F018111DACF21C0689431F8689432F840
:1069B000F2CF689433F8EFCF689434F8ECCFEAE084
:1069C0002E9E200D1124222E689435F8E4CF8E32AD
:1069D00029F436FC04C1689436F8DDCF8C3619F4FE
:1069E000689437F8D8CF8836B1F2982F9F7D9554A8
:1069F0009330E0F08336A1F18337C1F1833509F09C
:106A000063C02801F2E04F0E511CF801C080D18014
:106A1000692D70E036FC02C06FEF7FEFC6010E9467
:106A200059364C01689437F882010AC00C5F1F4F39
:106A3000FFE3F98388248394912C6501E89437F867
:106A400033FE2DC0522C8114910471F5552009F4A8
:106A500068CFB70180E290E00E946F365A94F6CF7B
:106A6000F801808189830E5F1F4FE4CF2801F2E097
:106A70004F0E511CF801C080D180692D70E036FCAA
:106A800002C06FEF7FEFC6010E9464364C018201A5
:106A9000D5CFB70180E290E00E946F362A94281487
:106AA000190409F0B0F7CECFF60137FC859137FE17
:106AB00081916F01B70190E00E946F3651105A9496
:106AC000F1E08F1A9108BFCF843619F0893609F0AA
:106AD00077C0F80137FE6BC060817181828193813C
:106AE0000C5F1F4FF32DFF763F2E97FF09C0909547
:106AF0008095709561957F4F8F4F9F4F689437F8C1
:106B00002AE030E0A5010E949F36C82ECA188C2CBE
:106B1000432C36FE0CC0E89440F8C91440F434FE0F
:106B200005C032FC03C0F32DFE7E4F2E892C44FE9F
:106B300095C0FE01EC0DF11D8081803309F087C006
:106B4000242D297E422E842D8870582E43FC95C01A
:106B500040FE8FC09C2C821418F42C0C922C981898
:106B600044FE91C0B70180E390E00E946F3642FE80
:106B700009C088E790E041FE02C088E590E0B701D7
:106B80000E946F36C91408F48AC0CA94D12C9FEFB2
:106B9000C91AD90ACA0CDB1CF60182916F01B70130
:106BA00090E00E946F36AC14BD04B1F74FCF608106
:106BB0007181072E000C880B990B0E5F1F4F92CF2F
:106BC000D32CE894D4F82AE030E0853739F1232D2E
:106BD000297FD22E8F3601F148F48835A9F0F701CC
:106BE000868197812B96E2E10C942F37803749F00C
:106BF0008837A9F7D4FE02C06894D2F820E130E0CB
:106C00000DC06894D4F8F6CF34FE03C0822F86609E
:106C1000D82E20E132E002C028E030E0F801D7FEB3
:106C20000FC060817181828193810C5F1F4FA5012C
:106C30000E949F36C82ECA183D2CE89437F867CFBB
:106C40006081718190E080E00E5F1F4FF0CF42FCC9
:106C500002C0839478CF8394839475CF842D8678F3
:106C600009F471CFF6CFB70180E290E00E946F3651
:106C700083948214C0F3512C73CF522C5818821471
:106C800008F46ECFF8CF842D867809F47BCF8BE2A1
:106C900041FE80E247FC8DE2B70190E071CFB70181
:106CA00080E390E00E946F369A946CCF8FEF9FEF55
:106CB00099CFFC010590615070400110D8F7809584
:106CC00090958E0F9F1F0895FC01615070400190B8
:106CD0000110D8F7809590958E0F9F1F08950F9300
:106CE0001F93CF93DF93182F092FEB018B8181FD29
:106CF00009C01FEF0FEF812F902FDF91CF911F91D0
:106D00000F91089582FF14C02E813F818C819D8157
:106D1000281739073CF4E881F981CF01019699835E
:106D2000888310838E819F8101969F838E83E3CF1A
:106D3000E885F985812F0995892BA1F3DACFFA012E
:106D4000AA27283051F1203181F1E8946F936E7FAA
:106D50006E5F7F4F8F4F9F4FAF4FB1E03ED0B4E09B
:106D60003CD0670F781F891F9A1FA11D680F791FDC
:106D70008A1F911DA11D6A0F711D811D911DA11DED
:106D800020D009F468943F912AE0269F11243019FD
:106D9000305D3193DEF6CF010895462F4770405D98
:106DA0004193B3E00FD0C9F7F6CF462F4F70405D47
:106DB0004A3318F0495D31FD4052419302D0A9F7A2
:106DC000EACFB4E0A6959795879577956795BA959C
:106DD000C9F700976105710508959B01AC010A2E62
:106DE00006945795479537952795BA95C9F7620F39
:106DF000731F841F951FA01D0895F999FECF92BDA2
:106E000081BDF89A992780B50895262FF999FECF6C
:106E10001FBA92BD81BD20BD0FB6F894FA9AF99AB7
:106E20000FBE019608952F923F924F925F926F92FC
:106E30007F928F929F92AF92BF92CF92DF92EF920A
:106E4000FF920F931F93CF93DF93CDB7DEB7CA1B8B
:106E5000DB0B0FB6F894DEBF0FBECDBF09942A88B6
:106E6000398848885F846E847D848C849B84AA845E
:106E7000B984C884DF80EE80FD800C811B81AA81EB
:106E8000B981CE0FD11D0FB6F894DEBF0FBECDBFB6
:106E9000ED0108955058BB27AA270E9462370C9431
:106EA000A5390E946C3938F00E94733920F039F40A
:106EB0009F3F19F426F40C9442390EF4E095E7FB59
:106EC0000C943C39E92F0E94CA3958F3BA1762076B
:106ED00073078407950720F079F4A6F50C94EC3934
:106EE0000EF4E0950B2EBA2FA02D0B01B9019001E5
:106EF0000C01CA01A0011124FF27591B99F0593F29
:106F000050F4503E68F11A16F040A22F232F342F70
:106F10004427585FF3CF469537952795A795F040BE
:106F20005395C9F77EF41F16BA0B620B730B840BD3
:106F3000BAF09150A1F0FF0FBB1F661F771F881F8B
:106F4000C2F70EC0BA0F621F731F841F48F48795E3
:106F500077956795B795F7959E3F08F0B0CF9395D5
:106F6000880F08F09927EE0F9795879508950E944E
:106F70006C3960F080E891E009F49EEF0E9473396B
:106F800028F040E851E071F45EEF0CC00C944239F7
:106F90000C94EC39E92FE0780E94CA3940F3092EAD
:106FA000052AB1F3261737074807590738F00E2E80
:106FB00007F8E02569F0E025E0640AC0EF6307F810
:106FC000009407FADB01B9019D01DC01CA01AD01A2
:106FD000EF930E944A380E94A5390E94FA375F91C8
:106FE000552339F02BED3FE049E450FD49EC0C947A
:106FF0004B370895DF93DD27B92FBF7740E85FE374
:107000001616170648075B0718F4D92F0E94F8399F
:107010009F938F937F936F930E943F3BECEAF0E046
:107020000E9445390E94A5392F913F914F915F9160
:107030000E94473ADD2351F09058A2EA2AED3FE042
:1070400049EC5FE3D0785D270E946237DF910C94B2
:10705000A5390E94183908F481E008950E947C390E
:10706000E3950C94B6390E9447380C94A5390E94D8
:10707000733958F00E946C3940F029F45F3F29F0D1
:107080000C943C3951110C94ED390C9442390E9406
:10709000CA3968F39923B1F3552391F3951B550B26
:1070A000BB27AA2762177307840738F09F5F5F4FDB
:1070B000220F331F441FAA1FA9F335D00E2E3AF01A
:1070C000E0E832D091505040E695001CCAF72BD032
:1070D000FE2F29D0660F771F881FBB1F2617370783
:1070E0004807AB07B0E809F0BB0B802DBF01FF27B5
:1070F00093585F4F3AF09E3F510578F00C943C391D
:107100000C94ED395F3FE4F3983ED4F38695779580
:107110006795B795F7959F5FC9F7880F911D96956D
:10712000879597F90895E1E0660F771F881FBB1FC9
:10713000621773078407BA0720F0621B730B840B76
:10714000BA0BEE1F88F7E09508950E94AC3868945A
:10715000B1110C94ED3908950E94D23988F09F57EF
:1071600098F0B92F9927B751B0F0E1F0660F771F6B
:10717000881F991F1AF0BA95C9F714C0B13091F061
:107180000E94EC39B1E008950C94EC39672F782F08
:107190008827B85F39F0B93FCCF386957795679526
:1071A000B395D9F73EF490958095709561957F4F92
:1071B0008F4F9F4F0895E89409C097FB3EF4909538
:1071C0008095709561957F4F8F4F9F4F9923A9F0C0
:1071D000F92F96E9BB279395F6958795779567954F
:1071E000B795F111F8CFFAF4BB0F11F460FF1BC093
:1071F0006F5F7F4F8F4F9F4F16C0882311F096E926
:1072000011C0772321F09EE8872F762F05C06623D3
:1072100071F096E8862F70E060E02AF09A95660F8C
:10722000771F881FDAF7880F9695879597F9089545
:10723000990F0008550FAA0BE0E8FEEF1616170687
:10724000E807F907C0F012161306E407F50798F0EF
:10725000621B730B840B950B39F40A2661F0232B08
:10726000242B252B21F408950A2609F4A140A69584
:107270008FEF811D811D089597F99F6780E870E069
:1072800060E008959FEF80EC0895DF93CF931F9304
:107290000F93FF92EF92DF927B018C01689406C0FE
:1072A000DA2EEF010E94473AFE01E894A59125915C
:1072B000359145915591A6F3EF010E946237FE0189
:1072C0009701A801DA9469F7DF90EF90FF900F9192
:1072D0001F91CF91DF91089500240A941616170686
:1072E00018060906089500240A94121613061406B7
:1072F000050608950C9442390E94D239D8F3E894D7
:10730000E0E0BB279F57F0F02AED3FE049EC06C0D4
:10731000EE0FBB0F661F771F881F28F0B23A620777
:107320007307840728F0B25A620B730B840BE39542
:107330009A9572F7803830F49A95BB0F661F771FC5
:10734000881FD2F790480C947F3B092E0394000CC1
:1073500011F4882352F0BB0F40F4BF2B11F460FFEF
:1073600004C06F5F7F4F8F4F9F4F0895EF93E0FFF3
:1073700007C0A2EA2AED3FE049EC5FEB0E946237CA
:107380000E94A5390F90039401FC9058E9EDF0E0BC
:107390000C94923B57FD9058440F551F59F05F3F96
:1073A00071F04795880F97FB991F61F09F3F79F027
:1073B00087950895121613061406551FF2CF4695A9
:1073C000F1DF08C0161617061806991FF1CF86952B
:1073D0007105610508940895E894BB27662777270F
:1073E000CB0197F908950E94183908F48FEF08959A
:1073F0009B01AC0160E070E080E89FE30C943338BF
:10740000FA01DC01AA0FBB1F9B01AC01BF5728F496
:10741000222733274427507820C0B75190F4AB2F50
:107420000024469537952795011CA395D2F300209B
:1074300071F0220F331F441FB395DAF30ED00C9472
:107440004A3761307105A0E88A07B94630F49B01DC
:10745000AC016627772788279078309621F0208323
:1074600031834283538308950E94473A0C94A5398F
:107470000E946C3938F00E94733920F0952311F086
:107480000C943C390C94423911240C94ED390E942F
:10749000CA3970F3959FC1F3950F50E0551F629F55
:1074A000F001729FBB27F00DB11D639FAA27F00D5D
:1074B000B11DAA1F649F6627B00DA11D661F829F84
:1074C0002227B00DA11D621F739FB00DA11D621F69
:1074D000839FA00D611D221F749F3327A00D611D86
:1074E000231F849F600D211D822F762F6A2F112468
:1074F0009F5750409AF0F1F088234AF0EE0FFF1F9B
:10750000BB1F661F771F881F91505040A9F79E3FF1
:10751000510580F00C943C390C94ED395F3FE4F355
:10752000983ED4F3869577956795B795F795E79547
:107530009F5FC1F7FE2B880F911D9695879597F950
:107540000895FA01EE0FFF1F309621053105A1F1D4
:107550006115710561F48038BFE39B0749F16894B8
:107560009038810561F08038BFEF9B0741F0992387
:107570004AF5FF3FE1053105210519F1E89408942A
:10758000E795D901AA2329F4AB2FBE2FF85FD0F3DA
:1075900010C0FF5F70F4A695E0F7F73950F019F0CE
:1075A000FF3A38F49F779F930DD00F9007FC9058C7
:1075B000089546F00C94423960E070E080E89FE363
:1075C00008954FE79F775F934F933F932F930E94C8
:1075D000E83B2F913F914F915F910E94343A0C9478
:1075E0004B3B9F930E947C390F9007FCEE5F0C94FD
:1075F000B63919F416F40C9442390C947D3B0E9470
:10760000D239B8F39923C9F3B6F39F57550B87FFC7
:107610000E948B3B0024A0E640EA900180585695DA
:10762000979528F4805C660F771F881F20F0261737
:107630003707480730F4621B730B840B202931296C
:107640004A2BA69517940794202531254A2758F7E9
:10765000660F771F881F20F026173707480730F47A
:10766000620B730B840B200D311D411DA09581F71A
:10767000B901842F9158880F9695879508959B019D
:10768000AC010C94343A29F416F00C943C390C9467
:10769000EC390C9442390E94D239A8F39638A0F7FD
:1076A00007F80F92E8942BE33AEA48EB5FE70E9471
:1076B0004A3A0F920F920F924DB75EB70F920E9407
:1076C000003AE7EFF0E00E9445394F915F91EF916A
:1076D000FF91E595EE1FFF1F49F0FE57E068442734
:1076E000EE0F441FFA95E1F74195550B0E94AA3B16
:1076F0000F9007FE0C94F83908959F3F31F0915098
:1077000020F4879577956795B795880F911D969585
:10771000879597F9089591505040660F771F881FFD
:10772000D2F708959F938F937F936F93FF93EF9377
:107730009B01AC010E94343AEF91FF910E944539C0
:107740002F913F914F915F910C94343A0C943C39B6
:107750000C947D3B0E94D239D8F39923C9F3940F3E
:10776000511DA3F39150504094F059F0882332F00A
:10777000660F771F881F91505040C1F79E3F5105FB
:107780002CF7880F911D9695879597F908955F3F7F
:10779000ACF0983E9CF0BB27869577956795B7959A
:1077A00008F4B1609395C1F7BB0F58F711F460FF6F
:1077B000E8CF6F5F7F4F8F4F9F4FE3CF0C94ED3932
:1077C00016F00C947D3B0C94423968940C943C392F
:1077D0000E94D239A8F39923C1F3AEF3DF93CF937C
:1077E0001F930F93FF92C92FDD2788232AF021973B
:1077F000660F771F881FDAF720E030E040E85FEB84
:107800009FE3883920F0803E38F021968F770E94E0
:107810004B37EFE1F1E004C00E944B37ECE4F1E0BC
:107820000E9445398B01BE01EC01FB2E6F57710997
:107830007595771F880B990B0E94DD3828E132E798
:1078400041E35FE30E94473AAF2D9801AE01FF90FC
:107850000F911F91CF91DF910E9462370C94A5394F
:10786000DB018F939F930E949B3CBF91AF91A29F9E
:10787000800D911DA39F900DB29F900D112408952E
:10788000AA1BBB1B51E107C0AA1FBB1FA617B70746
:1078900010F0A61BB70B881F991F5A95A9F7809562
:1078A0009095BC01CD010895A1E21A2EAA1BBB1B25
:1078B000FD010DC0AA1FBB1FEE1FFF1FA217B307BC
:1078C000E407F50720F0A21BB30BE40BF50B661FD2
:1078D000771F881F991F1A9469F760957095809596
:1078E00090959B01AC01BD01CF010895052E97FB3A
:1078F0001EF400940E948D3C57FD07D00E94543C1A
:1079000007FC03D04EF40C948D3C50954095309577
:1079100021953F4F4F4F5F4F0895909580957095FB
:1079200061957F4F8F4F9F4F0895EE0FFF1F05907A
:10793000F491E02D09940E94883DA59F900DB49F7D
:10794000900DA49F800D911D11240895B7FF0C94F4
:107950009B3C0E949B3C821B930B0895DF93CF932B
:107960001F930F939A9DF02D219FF00D8B9DF00D8D
:107970008A9DE02DF10D039FF00D029FE00DF11D9A
:107980004E9DE00DF11D5E9DF00D4F9DF00D7F931E
:107990006F93BF92AF925F934F93D5010E94883D42
:1079A0008B01AC01D7010E94883DEB01E80FF91F64
:1079B000D6010E94FD3C2F913F91D6010E94883D47
:1079C000C60FD71FE81FF91FAF91BF910E94FD3C62
:1079D0002F913F910E94883DC60FD71FE81FF91FC6
:1079E000D6010E94883DE60FF71F9801BE01CF0126
:1079F0000F911F91CF91DF9108950E94883D460F0E
:107A0000571FC81FD91F08F43196089597FB57FFD9
:107A10000C94163D9F938F930E94163D6E1B7F0B17
:107A2000AF91BF918A0B9B0B0895E894DF93CF939E
:107A3000FC01DB010E94883D7F936F93E9019A016D
:107A4000AC01BF93AF933F932F93DF010E94883D1A
:107A500026F46C1B7D0B820B930B9E01EB01FC014A
:107A60000E94FD3CAF91BF912F913F910E94FD3C40
:107A7000BE01CF01F9012F913F91CF91DF91089580
:107A8000002E083090F0982F872F762F652F542FD7
:107A9000432F322F22270850F4CF220F331F441FC9
:107AA000551F661F771F881F991F0A95B2F7002D73
:107AB000089597FD1094002E083098F00850232F59
:107AC000342F452F562F672F782F892F912DF4CFE4
:107AD0001594979587957795679557954795379519
:107AE00027950A95AAF71124002D08952A0D3B1D0C
:107AF0004C1D5D1D6E1D7F1D801F911F08952A194D
:107B00003B094C095D096E097F09800B910B0895B3
:107B1000A29FB001B39FC001A39F700D811D1124CE
:107B2000911DB29F700D811D1124911D0895FB01BF
:107B3000DC0102C001900D9241505040D8F70895E9
:107B4000DC0101C06D9341505040E0F70895FB0106
:107B5000DC018D91019080190110D9F3990B0895E2
:047B6000F894FFCFC7
:107B6400FFFFFFFF00E100000000000000005904D7
:107B740080000012131415161718191A1B1C1D0067
:107B8400070B0E0F00000000C40C770CAE0CF10CB8
:107B9400F10C00C1808100000000000000A806D79D
:107BA40008C906BE06E906CD06D90600000000E1B4
:107BB40009B409100A8A09AD099A098B09202035EC
:107BC40000313078006465006D41680073696E6748
:107BD4006C65730064696666004D55490025200094
:107BE400564F4C5400534348414C5445520047505F
:107BF400524D4300474E524D4300475047474100C2
:067C0400474E4747410016
:00000001FF
